:020000040800F2
:10000000789F0020810200088F630008894F000854
:100010008D6300082D0A0008E97100080000000047
:10002000000000000000000000000000A101000826
:10003000BB0F000800000000FD010008956A0008E1
:100040009B0200089B0200089B0200089D680008B4
:100050009B0200089B0200089B0200089B0200080C
:100060009B0200089B0200089B0200089B020008FC
:100070009B0200089B0200089B0200089B020008EC
:100080005D0F0008690F00089B020008490A00087C
:10009000310A00089B0200083D0A00089B02000884
:1000A0009B0200089B0200089B0200089B020008BC
:1000B0009B02000800000000000000009B020008F6
:1000C0009B0200089B0200089B0200089B0200089C
:1000D0009B0200089B020008B97100089B020008FF
:1000E0009B0200089B0200080000000000000000C6
:1000F0000000000000000000000000000000000000
:10010000000000009B020008000000009B020008A5
:100110000000000000000000516B00089B02000876
:100120009B0200089B0200089B0200089B0200083B
:100130009B0200080000000000000000000000001A
:100140009B0200089B0200089B02000800000000C0
:10015000750F0008810F00089B0200089B02000831
:100160009B0200089B0200089B02000800000000A0
:100170009B0200089B020008000000000000000035
:100180009B0200089B0200089B020008DFF80CD0CD
:1001900000F03AFC00480047B18A0008789F002030
:1001A0002C4B1968086800F05AB880F30988BFF32F
:1001B0006F8F4FF0000080F311887047000000003F
:1001C00008480068006880F308884FF0000080F35A
:1001D000148862B661B6BFF34F8FBFF36F8F00DF35
:1001E00000BF00BF08ED00E0DFF80C00016841F43B
:1001F00070010160704700BF88ED00E0EFF30980F7
:10020000BFF36F8F134B1A681EF0100F08BF20ED5D
:10021000108A20E9F04F106009B44FF0500080F3CD
:100220001188BFF34F8FBFF36F8F09F0E3FC4FF0DE
:10023000000080F3118809BC1968086800F014B840
:100240001EF0100F08BF00F014B880F30988BFF348
:100250006F8F70478C000020EFF30580704730C827
:10026000B0E8C04FFFF7A1BF30C8B0E8C04FFFF7FC
:10027000E7BFB0EC088AB0EC08CAFFF7E6BF0000A1
:100280000648804706480047FEE7FEE7FEE7FEE730
:10029000FEE7FEE7FEE7FEE7FEE7FEE7416B00084C
:1002A0008D0100082DE9F05F0546002092469B462F
:1002B00088460646814640241BE02846414647467C
:1002C000224600F053FA53465A46C01A914110D3C1
:1002D00011461846224600F03AFA2D1A67EB01083B
:1002E0004F4622460120002100F031FA17EB0009A9
:1002F0004E41201EA4F10104DFDC484631462A4667
:10030000434600F000B830BCBDE8C09F40EA01039E
:100310009B0703D009E008C9121F08C0042AFAD2BB
:1003200003E011F8013B00F8013B521EF9D270477F
:10033000D2B201E000F8012B491EFBD27047002227
:10034000F6E710B513460A4604461946FFF7F0FFD4
:10035000204610BD421C10F8011B0029FBD1801A59
:1003600070472DE9FE4F804681EA0300C00F0C461E
:10037000009021F0004123F00045B8EB0200A941B4
:1003800005D24046214690461C460B46024623F0C5
:100390000040104347D0270DC7F30A00C3F30A51AA
:1003A0000290401A019040286BDAC3F3130040F426
:1003B000801B0098924620B10023D2EB030A63EB26
:1003C0000B0B01985946C0F14002504600F0BFF9AE
:1003D00006460D4650465946019A00F0D7F910EBF3
:1003E00008006141002487EA115284EAE7731A4346
:1003F00040D0009A62B3019A012A4FEA075215DCF5
:10040000001B61EB02014FF0004202EA0752CDE906
:100410000042001C41F5801132462B4600F00EFAD6
:1004200003B000F045B840462146F9E7001B61EBF8
:100430000201001C41F5801300185B412018A2F551
:10044000001747EB030140EAD570B6196D4111E082
:100450006D084FEA360645EAC0754FEA0752001BA1
:1004600061EB0201001C41F5801149084FEA3000A0
:100470000019514132462B4603B000F01CB800F081
:10048000CEB90098012240000023D0EB020263EBBA
:10049000E073009821464FEAE074B8EB000061EB8E
:1004A0000401E9E783F000435BE781F0004158E78E
:1004B00030BCBDE8C08F30BCBDE8C04FFFF7DFBF28
:1004C0002DE9FE4F81EA030404F0004421F00041CD
:1004D00000944FF0000B23F0004350EA01045ED07B
:1004E00052EA03045BD0C3F30A54C1F30A552C4407
:1004F000A4F2F3340194A0FB0254C1F3130141F4BC
:100500008011C3F3130343F4801301FB024400FB87
:10051000034E840A970A44EA815447EA8357A4FBAE
:10052000076802958D0A05FB07854FEA932C04FBAB
:100530000C542705029D4FEA065847EA1637B5EBDB
:1005400008056EEB070C870E920E47EA811742EA08
:100550008312A7FB0201B6EB0B0164EB00042B0D29
:1005600043EA0C335E1844EB1C50DA465146E7FB75
:100570000201C5F313044FEA0B3343EA14534FEA65
:100580000432019C43EA0603A4F10C040294009C8B
:10059000CDE900B400F052F903B000F003B8002038
:1005A0000146F9E730BCBDE8C08F2DE9F04D81EA86
:1005B000030404F0004B21F0004514464FF0000AFC
:1005C00023F0004150EA050220D054EA01021DD078
:1005D000C5F30A570246C5F31303C1F31300C1F371
:1005E0000A5640F4801543F48013A7EB0608101B4D
:1005F000D64608F2FD3873EB050002D308F1010876
:1006000001E092185B41B8F1000F03DA00200146C7
:10061000BDE8F08D00204FF48011064684460EE0C0
:10062000171B73EB050705D3121B63EB050306438A
:100630004CEA010C49084FEA300092185B4150EA3D
:100640000107EDD152EA030012D082EA040083EAE6
:100650000501084305D0101BAB4106D2012200233F
:1006600006E000224FF0004302E06FF00102531059
:100670001AEB06004CEB085110EB0A0041EB0B01A2
:10068000BDE8F04D00F0CBB80EB5C10F80EAE070C8
:100690000844CA07002140F233438DE80E000A46A1
:1006A0000B4600F0CBF803B000BD0EB540F233416D
:1006B00002910021CDE900110A460B4600F0BEF878
:1006C00003B000BD00F0004230F000400AD0C10D80
:1006D00001F56071C0F3160042EA0151C2084007FB
:1006E0001143704700200146704701F0004330B4C9
:1006F00021F0004150EA010206D00A0DA2F5607215
:10070000C1F31301002A02DC30BC00207047440F03
:1007100044EAC104C100E01830BC00EBC25000F054
:1007200047B830B50B46014600202022012409E0DD
:1007300021FA02F59D4205D303FA02F5491B04FA9A
:1007400002F52844151EA2F10102F1DC30BD202A79
:1007500004DB203A00FA02F1002070479140C2F118
:10076000200320FA03F3194390407047202A04DB4A
:10077000203A21FA02F00021704721FA02F3D0401A
:10078000C2F120029140084319467047202A06DB37
:10079000CB17203A41FA02F043EAE07306E041FA4F
:1007A00002F3D040C2F1200291400843194670473D
:1007B0000029A8BF7047401C490008BF20F0010075
:1007C000704710B4B0FA80FC00FA0CF050EA010453
:1007D00004BF10BC704749B1CCF1200421FA04F4E5
:1007E00011FA0CF118BF012121430843A3EB0C01BE
:1007F000CB1D4FEA00614FEA102042BF002010BC21
:10080000704700EBC35010440029A4BF10BC7047D0
:10081000401C490008BF20F0010010BC704710B513
:10082000141E73F1000408DA401C41F10001921813
:100830005B411A4301D120F0010010BD2DE9F04DBC
:1008400092469B4611B1B1FA81F202E0B0FA80F211
:1008500020329046FFF77BFF04460F4640EA0A002D
:1008600041EA0B0153465A46084313D0114653EA56
:10087000010019D0C8F140025046FFF777FF054646
:100880000E46504659464246FFF761FF084305D0E1
:10089000012004E020463946BDE8F08D00200543E4
:1008A00046EAE0762C4337430A986305E40AA0EB56
:1008B00008000022FD0A44EA47540A3002D500200D
:1008C0000146E9E7010510196941DDE9084500190C
:1008D0006941BDE8F04DA2E770B521F00043034344
:1008E0000CD0C1F30A550024D5EB040564EB0403D6
:1008F000D617AD1AB34102DB0020014670BD2018A7
:1009000041EB025170BD2DE9F04D00231A461B1A30
:100910008A4103DB00200146BDE8F08DC1F30A5295
:10092000C1F3130141F480154FF0000BD10702D140
:1009300000186D41521E0027044640F2FF11384650
:1009400001EB620A3E468046024600204FF48011C9
:10095000FFF70CFFC2197141BB1846EB0100B4EB65
:10096000030C75EB000C04D3E41A65EB0005174685
:100970000E46241908F101006D4180463428E3DD5C
:10098000F91946EB0600091BA84103D24FF0FF32CC
:10099000134601E0002213461BEB070046EB0A5109
:1009A000BDE8F04DFFF73BBFC1F30A52C1F313019D
:1009B00040F2FF3341F480119A4202DA00200146EE
:1009C000704740F233439A42A2F2334202DC524271
:1009D000FFF7CCBEFFF7BBBE30B5041E71F10004BB
:1009E00004DB4FF00044404264EB0101141E73F13C
:1009F000000405DB1C464FF00043524263EB040346
:100A0000994208BF904230BD064C074D06E0E068B1
:100A100040F0010394E8070098471034AC42F6D345
:100A2000FFF7B8FB5CA900087CA90008FEE70000FE
:100A3000014801F0FBBC0000106A0020014801F0F1
:100A4000F5BC0000106A0020014801F0EFBC000076
:100A5000106A002070B506461D480D46006883697F
:100A60001A0EC3F30741580730D51A4C607838B9CD
:100A700019A006F0BBFB0120607002F09FFB6061D3
:100A800002F09CFB6169401AB0F57A7F17D91FA06C
:100A900006F0ACFB0E4801F091FF0D4801F03BFC65
:100AA00005F00AFB0A4801F05DFF40F202410848E8
:100AB00001F049FB1FA006F099FB002060700A219D
:100AC000304608F0C3FF2868401C286070BD000055
:100AD000106A002010000020205B43414E20455248
:100AE000524F525D204275732D4F666620646574C7
:100AF00065637465642120544543203D2025642CA2
:100B000020524543203D2025640A00005B43414EAE
:100B10005D2052657374617274696E672043414E43
:100B2000206166746572204275732D4F66662E2EA5
:100B30002E0A00005B43414E5D2043414E2072650A
:100B400073746172746564206166746572204275A5
:100B5000732D4F66660A000030B58BB0002001246B
:100B6000CDE906040590049080200425CDE9000518
:100B70004FF6FF7008940290039069460F4801F009
:100B800053FB40B988200594CDE9000569460B4820
:100B900001F04AFB20B100F053FA01200BB030BD48
:100BA000064801F044FD0028F8D0044801F0C8FBD5
:100BB000014603A006F01AFBEDE70000106A0020D2
:100BC00043414E20496E697469616C697A61746948
:100BD0006F6E204572726F723A20256C640A0000B5
:100BE00030B587B01206DDE90A45120942EA033240
:100BF00004F00F0342EA032205F00F0342EA031256
:100C000042F080520192042202920022CDE9032197
:100C1000024606AB6946074801F0A7FA010007D073
:100C200005A006F0E3FA0348416A10A006F0DEFAD8
:100C300007B030BD106A002048414C5F43414E5F11
:100C400041646454784D65737361676520666169BA
:100C50006C6564202C207265745F737461747573A5
:100C60003A30782578200D0A000000006863616E34
:100C70002D3E4572726F72436F64653A203078255D
:100C800078200D0A00000000F0B589B00024DDE9ED
:100C90000E560094019417788DF8007057788DF8EF
:100CA000017097788DF80270D278000600098DF8EF
:100CB000032040EA033005F00F0240EA022006F06C
:100CC0000F0240EA02100390042004900194CDE941
:100CD000054108AB6A4602A9074801F046FA01003F
:100CE00007D006A006F082FA0348416A10A006F079
:100CF0007DFA09B0F0BD0000106A002048414C5F49
:100D000043414E5F41646454784D65737361676518
:100D1000206661696C6564202C207265745F737451
:100D2000617475733A30782578200D0A0000000050
:100D30006863616E2D3E4572726F72436F64653AEF
:100D40002030782578200D0A00000000F0B587B02B
:100D50000D460746DDE90C101206120942EA03327D
:100D600001F00F0142EA012100F00F0041EA0010FA
:100D70000190042002900020CDE9030506AB3A461D
:100D80006946134801F0F1F920B112A006F02EFADD
:100D900007B0F0BD05EB450007F0EAFE064600246B
:100DA0000AE000BF04EB440037F81420304410A1DF
:100DB00006F02CFA641CE4B2AC42F3D332460EA027
:100DC000019906F013FA304607F04AFEE0E700000A
:100DD000106A002043414E206D6573736167652082
:100DE00073656E64206661696C65640A00000000CA
:100DF000253032582000000043414E206D6573734A
:100E00006167652073656E743A2049443D307825EA
:100E10003038582C20446174613D25730A0000006D
:100E20002DE9FC41044601200225CDE900500E4E7B
:100E30000F462378B288082106F12C00FFF7D0FE78
:100E4000009501952378B288082106F13400FFF758
:100E5000C7FE002007F0E4FD2078401C2070002031
:100E60003860BDE8FC81000010000020411A01F14B
:100E700021026FF00500032A06D34A1C032A03D37C
:100E80001F39032900D3002070470A2007F0A6FE6F
:100E9000FBE7000070B586B014216846FFF74FFAF3
:100EA0002C4C54F84C0F40F001002060206800F0FA
:100EB00001000590206840F002002060206800F0EA
:100EC00002000590606C40F400406064E06840F40B
:100ED0000030E060E0684FF0904500F4003005908D
:100EE00003200190002002904FF6FF7000906946A9
:100EF000284602F073F847F6FF70174E00906946D7
:100F0000304602F06BF801224FF4F051284602F00F
:100F100050F9012248F20101304602F04AF900225C
:100F20001021304602F045F9206820F001002060D1
:100F3000206820F002002060E06820F40030E060CB
:100F4000E06820F40010E060E06820F00070E060ED
:100F500006B070BD0010024000040048014801F0D6
:100F6000B0BD0000C46B0020014801F0AABD000024
:100F70000C6C0020014801F0A4BD00008C6A002028
:100F8000014801F09EBD0000D46A002030B590F801
:100F9000444004F01C050124AC40056C6C600468FE
:100FA00063608368102B036803D099600068C26097
:100FB00030BD9A600068C16030BD704770B50446AE
:100FC000074803F0FDF9A4F109050422214604486D
:100FD00003F03CFA2946BDE8704002A006F006B9CD
:100FE0001C6B00205254432057616B657570205470
:100FF000696D65722073657420666F7220256420A8
:10100000730A000010B509A006F0F0F8FFF742FFE0
:101010000A488078FFF7D2FF4FF4806002F02AFC84
:10102000BDE81040012002F059BC0000456E746517
:1010300072696E672053746F70320A0016000020C8
:1010400072B6FEE72DE9F04F04462DED068BBDB0DC
:101050008846B0F84000C0F303113B91C0F3032170
:101060003A911E2101EB1036B4F842B000F00F07A0
:10107000002220A904EB42009300B0F84400521C67
:1010800000F00F0541F8235001EB8303C0F3031573
:101090005D60C0F30325000BC3E90250062AE9DBBB
:1010A0005FF0000051F82020072A02DD103A41F8D5
:1010B0002020401C1828F5DB00206A4604EB400382
:1010C0008500B3F85030401C03F00F0C42F825C0E7
:1010D00002EB8505C3F3031CC5F804C0C3F3032C5E
:1010E0001B0BC5E902C30828E8DB002052F82030BA
:1010F000072B02DD103B42F82030401C2028F5DB96
:10110000012000FA07FA0025DFED658A3046FFF777
:10111000CCFA9FED649BB6EE008ACDE9380108F564
:101120002059002707EB451004EB4001B1F880106F
:10113000C1F3051100EE101A5C49B8EE401A01EB3C
:1011400080065B4911EE100A86ED001A884205DD23
:101150009FED580A31EE400A86ED000A20A83A9920
:1011600050F8250000EE10AA884000EB0B02B8EE04
:10117000C00AD6ED000A5DF827003B9920EE800AF0
:101180008840104400EE900AF8EEE00A30EE800A43
:10119000F0EE690A86ED000ADDE9380141EC110B39
:1011A000B0EE490A06F080F8B0EE40AAF0EE60AA70
:1011B0003068FFF787FA53EC1A2BFFF7F6F9FFF7C1
:1011C00094FA01EE100A7F1C86ED001A99ED960A3A
:1011D000D9ED970A202F30EE200AD8ED060A20EE2E
:1011E000200A00EE481A88EE810A86ED000A99DB93
:1011F0006D1C182D95DB2D4D01204FF4407795ED9A
:10120000001A00BF05EB800191ED000AB4EEC10A9F
:10121000F1EE10FA01DDB0EE401A401CB842F1DBED
:101220000024B0EE000A4FF08E4103E021EE001AD8
:10123000641CE4B211EE100A8842F7DB0026204657
:10124000FFF733FA8A468146B0EE49AAF0EE69AA62
:101250004AEC119BB0EE4A0AF0EE6A0A06F024F856
:10126000B0EE409AF0EE609A55F82600FFF72AFAA1
:1012700053EC192BFFF724F9FFF737FA00EE100AA9
:1012800008EB8600761C30EE080ABE4280ED130A99
:10129000DEDB88F84C4C3DB0BDEC068B00F00CB8A2
:1012A000BD37863500000000000000401C01002012
:1012B0000000F8410000804230BCBDE8C08F000053
:1012C00010B5828A802303EA121282F08003B0F8FC
:1012D0006A20204C02F03F0000EE100AB8EE400AEF
:1012E00010EE100AA04203DDDFED1B0A30EE600AAB
:1012F000DFED1A0AC2F38410194C60EE200A00EEEA
:10130000100A9FED181AB8EE400A10EE100AA0421B
:1013100001DD30EE410AF6EE001AD00A60EE211A25
:1013200000EE100AB8EE400A10EE100AA04201DDED
:1013300030EE410AB4EE001A81F8253001F5205153
:1013400020EE010AC1ED990AC1ED9A1A81ED9B0ABE
:1013500010BD00000000F841000080420000803D08
:1013600000007041000000422DE9F04106462DEDDD
:10137000088B0D461B21B0F84000B6F8742001EB35
:101380001031C2F3090060F30F04B0F5007F03DBF6
:10139000A0F5806060F30F04900A60F31F441F28DB
:1013A00002DD403860F31F4404EB244060F31F4427
:1013B000B6F87200594AC0F3090000EE100AB8EE00
:1013C000408A18EE100A904203DD9FED550A38EE70
:1013D000408A0846FFF769F941EC110B9FED519BDC
:1013E000B0EE490AF0EE690A05F05EFFB0EE401A71
:1013F000F0EE601AB0EE41AAF0EE61AA18EE100A03
:10140000FFF760F953EC1A2BFFF7CFF8FFF76DF9F0
:1014100001EE900AB6F8720011EE907A800A00EEA2
:10142000100A4249B8EE401A11EE100A884203DD54
:101430009FED3F0A31EE401ADFED3E0AB7EE000A9B
:1014400096F8760001EE200ADFF8EC809FED3BAACB
:1014500060EE218A00EE100AB8EE408A18EE100AFB
:10146000404501DD38EE4A8A96F87000C0F303105B
:101470000830FFF71AF941EC110BB0EE490AF0EE13
:10148000690A05F011FFB0EE40BAF0EE60BA18EE4E
:10149000100AFFF717F953EC1B2BFFF786F8FFF73D
:1014A00024F92862B6F87600000A00EE100AB8EEB9
:1014B000408A18EE100A404501DD38EE4A8AB6F837
:1014C0007000C0F30320FFF7F0F841EC110BB0EE11
:1014D000490AF0EE690A05F0E7FEB0EE409AF0EE38
:1014E000609A18EE100AFFF7EDF853EC192BFFF78E
:1014F0005CF8FFF7FAF8E86105F5205005F50055AE
:10150000C0F85872C0ED978AA5F8604A2014A5F873
:10151000620ABDEC088BBDE8F08100000080FF434B
:101520000000804400000000000000400000F8417E
:10153000000080420000003C0000FE4200008043AA
:101540002DE9F0410E46002107460C460D4608469F
:101550004FF6FF7306EB410202F50052491CA2F858
:10156000703A89B2A2F87A3A0529F3D300214FF4F0
:10157000407300BF07EB4102B2F88020BAB1D20736
:1015800007D006EB450202F500526D1CA2F87A1A4C
:10159000ADB2491C89B2994203D2052C01D2052D66
:1015A000E8D3042C0CD96FF00200BDE8F08106EB03
:1015B000440202F50052641CA2F8701AA4B2E8E7D3
:1015C000042D02D96FF00300EFE76119042902D955
:1015D0006FF00400E9E7002317E006EB43015F1C0E
:1015E00001F500580DE000BF06EB470000F5005084
:1015F000B0F8701AB8F8700AFFF738FC0028D4D198
:101600007F1CA742F0DB5B1C9BB2A342E5D3002307
:1016100017E006EB43015F1C01F500580DE000BF29
:1016200006EB470000F50050B0F87A1AB8F87A0ACD
:10163000FFF71CFC0028B8D17F1CAF42F0DB5B1C1D
:101640009BB2AB42E5D3002317E006EB4301002732
:1016500001F500580DE000BF06EB470000F5005013
:10166000B0F87A1AB8F8700AFFF700FC00289CD18D
:101670007F1CAF42F0DB5B1C9BB2A342E5D394E737
:10168000B0F96000B0F5004F00DB00B2888270470F
:10169000B0F878000A4A000A00EE100AB8EE400AD4
:1016A00010EE100A904203DDDFED060A30EE600A0C
:1016B000DFED050A20EE200A81ED0A0A70470000DE
:1016C0000000FE42000080430000003930B530F8D1
:1016D0007E2F6FF02703C2F3013202EB8202520029
:1016E000A1F840300023A1F8423010F80439C3F3C8
:1016F0000313A1F844308488C4F3032413FB02F3DA
:10170000A1F8443014FB0232A1F846204FF4C8720D
:10171000A1F848200279224D02F00F03012208337C
:101720009A400378DFED1F0A00EE103AB8EE400A47
:1017300081ED0B0A03881B0A00EE103AB8EE400A4E
:1017400081ED0C0A837800EE103AB8EE400A81ED84
:101750000D0A4088000A00EE100A0020B8EE400A88
:1017600081ED0E0A01EB800393ED0B0A10EE104A97
:10177000AC4203DD30EE600A83ED0B0AB0EE401A96
:1017800000EE102A401C0428B8EEC00AC1EE001A70
:10179000C3ED0B1AE6DB9FED040A81ED0F0A30BDA5
:1017A0000000FE420000804317B751B92DE9F34F06
:1017B00006462DED068B83B0B0F86C1041F3072080
:1017C0007F2800DD40B28DF8080048B27F2800DD98
:1017D00040B28DF80A00B6F86E1041F307207F285A
:1017E00000DD40B28DF8090048B27F2800DD40B22C
:1017F0008DF80B0096F870100025C1F3031001F06E
:101800000F02012101FA02F8DFF8A8A10DF1080B7F
:10181000DFF8A4910830FEF748FF9FED688BCDE913
:101820000001002404EB4511C81701EBD06201EB65
:10183000906080115211404202EB400001EBD172E6
:1018400022F001028A1A02EB4000C2B206EB41000C
:1018500009EB810790F88000C0F3420000EE100A07
:10186000B8EE401A11EE100A87ED001A504505DD5A
:10187000B2EE000A31EE400A87ED000A00EE108A4F
:10188000D7ED000A1BF90200B8EEC00A20EE800A6C
:1018900000EE900AF8EEE00A30EE800AF0EE680AF8
:1018A00087ED000ADDE9000141EC110BB0EE480ABA
:1018B00005F0FAFCB0EE401AF0EE601AB0EE419A74
:1018C000F0EE619A3868FEF7FDFE53EC192BFEF737
:1018D0006CFEFEF70AFF641C3860202CA2DB6D1C36
:1018E000182D9EDB99ED000A4E460120B0EEC01A7D
:1018F0004FF4407706EB800191ED000AB0EEC00A8C
:10190000B4EEC10AF1EE10FA01DDB0EE401A401C4F
:10191000B842EFDB0025B0EE000A4FF0854103E04E
:1019200021EE001A6D1CEDB211EE100A8842F7DBB1
:1019300000242846FEF7B9FE89468046B0EE489A54
:10194000F0EE689AB6EE00AA49EC118BB0EE490AA7
:10195000F0EE690A05F0A8FCB0EE408AF0EE608A6D
:1019600056F82400FEF7AEFE53EC182BFEF7A8FD48
:10197000FEF7BBFE00EE100AB5EEC00AF1EE10FA5B
:1019800002D230EE4A0A01E030EE0A0A0A9800EB71
:10199000840000F58050641C80ED940ABC42D3DBC7
:1019A0000A9800F5805080F8505E03B0BDEC068BBD
:1019B00000F008B8000040401C0D002000000000AE
:1019C000000000401CBCBDE8E08F00002DE9F04F96
:1019D00089462DED068B81B0B0F86820110B0729E0
:1019E00000DD10398DF80010C2F30321072900DD56
:1019F00010398DF80210C2F30311072900DD1039E8
:101A00008DF8011002F00F01072900DD10398DF863
:101A10000310B0F870000025C0F30320E846544ED0
:101A2000FEF743FE8B4682469FED528B5FF000042B
:101A300004EB4510C11700EBD16200EB91618911F5
:101A40005211494202EB410100EBD07222F0010237
:101A5000821A02EB4101C9B218F9011006EB8007A6
:101A600000EE101A4BEC11ABF0EE680AB8EEC00AAB
:101A700087ED000AB0EE480A05F016FCB0EE409A79
:101A8000F0EE609A3868FEF71DFE53EC192BFEF756
:101A90008CFDFEF72AFE641C3860202CC8DB6D1C10
:101AA000182DC3DB96ED000A01204FF44077B0EE0D
:101AB000C01A00BF06EB800191ED000AB0EEC00A2B
:101AC000B4EEC10AF1EE10FA01DDB0EE401A401C8E
:101AD000B842EFDB0025B0EE000A4FF0854103E08D
:101AE00021EE001A6D1CEDB211EE100A8842F7DBF0
:101AF00000242846FEF7D9FD8A468046B0EE489A73
:101B0000F0EE689AB6EE00AA4AEC118BB0EE490AE4
:101B1000F0EE690A05F0C8FBB0EE408AF0EE608A8C
:101B200056F82400FEF7CEFD53EC182BFEF7C8FC48
:101B3000FEF7DBFD00EE100AB5EEC00AF1EE10FA7A
:101B400002D230EE4A0A01E030EE0A0A09EB8400C4
:101B500000F5E050641C80ED950ABC42D4DB42F6EF
:101B6000542000F8095001B0BDEC068B00F006B817
:101B70001C190020000000000000004030BCBDE83F
:101B8000C08F00002DE9F04F8B46018CB0F9224048
:101B9000B8B001F00F09C1F3031CC1F3032AB4F577
:101BA000004F00DB24B2002120AA00EB41038D008E
:101BB0009B8C491C03F00F0642F8256002EB85055B
:101BC000C3F303166E60C3F303261B0BC5E9026360
:101BD0000629EADB5FF0000152F82130072B02DD15
:101BE000103B42F82130491C1829F5DB00236946D7
:101BF00000EB43059E002D8E5B1C05F00F0741F89E
:101C0000267001EB8606C5F303177760C5F303273B
:101C10002D0BC6E90275082BEADB002351F823508F
:101C2000072D02DD103D41F823505B1C202BF5DB16
:101C30000023964600225EF8235005FA0AF500BFFD
:101C400002EB431600EB46070BEB4606B7F8807035
:101C5000BF0AA6F84E7C1F2F02DD403FA6F84E7C3F
:101C600031F82280BFB207FA09F708FA0CF8A84445
:101C700027444744521CA6F84E7C202AE0DB5B1C1C
:101C8000182BD7DB38B000F000B830BCBDE8C08FEF
:101C900070B50C462DED048B0546B0F86410254A4E
:101CA000880A00EE100AB8EE400A10EE100A9042C0
:101CB00003DDDFED210A30EE600ADFED200AC1F31B
:101CC00009001F4920EE208A00EE100AB8EE400AF3
:101CD00010EE100A884203DDDFED1A0A30EE600ACA
:101CE000F4EE000AB5F862609FED171B60EE208AE3
:101CF0009FED170B05F0D8FA288CB0EE409AF0EE65
:101D0000609A00F47040FEF7D0FC53EC192BFEF7FC
:101D10004CFC9FED111B53EC112BFEF722FBFEF741
:101D2000E4FC84ED018AC4ED028AA6812061BDEC49
:101D3000048B70BD0000F841000080420000803933
:101D40000080FF43000080440000000000002C40A1
:101D500000000000000000400000000000002040E3
:101D600090F87800094A00EE100AB8EE400A10EE2A
:101D7000100A904203DDDFED060A30EE600ADFED67
:101D8000050A20EE200A81ED060A70470000FE4297
:101D9000000080430000003D10B5B0F866300A4AEC
:101DA000180A7F28108002DDA0F5807010800004E2
:101DB000C00ADBB24FF44044108004EB431353805D
:101DC00008805088488010BD00000020144A117F10
:101DD0001448012901D003290FD1036823F40073AB
:101DE0000360036843F400630360036823F4006343
:101DF0000360036843F400730360022901D00329E0
:101E00000BD1016841F480510160016821F48051D7
:101E10000160016841F48061016000201077704723
:101E20006800002000200240C107054803D0416936
:101E300041F004014161416941F4803141617047E1
:101E40000020024008494A69C0B222F47E7242EA88
:101E5000C0004861486940F002004861486940F4A8
:101E6000803048617047000000200240054910B5ED
:101E70004C6944F001044C610260BFF36F8F436012
:101E800010BD000000200240094A10B554694023EB
:101E900044F480245461EFF3108272B610C910C06C
:101EA0005B1E13F0FF03F9D182F3108810BD000010
:101EB0000020024070B5054601F080F90646134C3B
:101EC00008E0681C06D001F079F9801BA84201D314
:101ED000032070BD2069C003F3D420690C49084079
:101EE0000CD00C494A6802434A60810F01D0A169B5
:101EF000A161810000D02061012070BD2069C00770
:101F000001D001202061002070BD000000200240AF
:101F1000FAC302006800002070B586B00C000546C8
:101F200028D01548854225D80026049600F0A0FF49
:101F30001248816941F0404181614CF2FA310161FE
:101F40002846009600F01CF80190284600F026F87C
:101F5000029005EB8400401E00F020F80299401A20
:101F6000401C039004A9684600F0B2FE002801D08E
:101F700000F01EFF06B070BD000004080020024003
:101F80000449096804494FF001000968CA43120472
:101F9000120C704700000140E075FF1F0E4910B59C
:101FA00009684FF48024CB431A04120C0AD00A04A7
:101FB0005FEA921202F10062824205D9A0F100604C
:101FC000C00A10BD2246F5E71A04120C01D009041C
:101FD0008C09001BF2E70000E075FF1F064B10B5EF
:101FE000984207D8002303E010F8014BCC545B1C47
:101FF0009342F9D310BD0000000004082DE9F04120
:1020000017460D46044600F033FF0F48844216D2AF
:10201000002609E0D5E900232146002000F0D2FE89
:1020200068B908340835761CB6EB570FF2D3F807B9
:1020300005D06368214600202A6800F0C3FEBDE891
:10204000F04100F0B5BE0000000004082DE9F04F9B
:10205000E5B0994614460E0083460CD0A1074FEA1E
:10206000940000D0401C00271FFA80FA8DF8007001
:102070003D46E8460CE0012065B000F031B8684606
:10208000FEF768F94044725D13A105F0BFF86D1CBE
:10209000A542F4D301215846FFF73EFF5246314690
:1020A0005846FFF7ABFF224649465846FFF796FFD2
:1020B0008DF8C870002532AE09E032A8FEF74AF963
:1020C000304419F8052004A105F0A0F86D1CA542C4
:1020D000F3D30020D0E70000253032582000000064
:1020E00030BCBDE8C08F70B500224D1E16E0531CF9
:1020F00000EB82040FE000EB8306D4ED000A96EDBE
:10210000000AB4EEE00AF1EE10FA03D284ED000A00
:10211000C6ED000A5B1C8B42EDDB521CAA42E6DBDB
:10212000CA0701EBD1714FEA610100EB810090ED2C
:10213000000A07D150ED010A30EE200AF6EE000A3F
:1021400020EE200A70BD90F82020012A07D0022A34
:1021500005D0416A41F48021416201207047006846
:1021600042690A43426100207047F0B590F8205060
:102170000468A468012D05D0022D03D0416A41F402
:1021800080214DE014F0406F01D1E50045D5C4F346
:1021900001640125A5401D608D684FF4C0739DB199
:1021A000CE6835434E6845EAC605066803EB04175A
:1021B000F5514FF4C275076805EB04150E697E51A1
:1021C000097D012905D009E00E88CD6845EA46550C
:1021D000EBE701684E5946F480764E511179D2F8FA
:1021E00005504FF4C67641EA0521056806EB041652
:1021F000A9511178D2F801204FF4C47541EA0221A7
:10220000026805EB04155151006803EB04114258B4
:1022100042F0010242500020F0BD416A41F4001139
:1022200041620120F0BD000010B590F82030026836
:10223000012B07D0022B05D0416A41F48021416275
:10224000012010BDD2F8000240F00100C2F80002E7
:10225000087D00F01F0301209840D2F81C32834310
:10226000C2F81C32CB69B3B9D2F80C328343C2F83E
:102270000C328C894B6864F31F434C6902EBC40435
:10228000C4F840320C890B6864F31F434C6902EBBD
:10229000C404C4F84432CB69012B16D1D2F80C32F5
:1022A0000343C2F80C320C884B6864F31F434C693B
:1022B00002EBC404C4F840320C89CB6864F31F43BA
:1022C0004C6902EBC404C4F844328B69002BD2F889
:1022D00004320FD053EA0003C2F804320B69002B1A
:1022E000D2F8143208D00343C2F81432096A012923
:1022F00004D008E08343EFE78343F5E7D2F81C12EC
:102300000143C2F81C12D2F8000220F00100C2F80A
:102310000002002010BD10B504000ED000F04EFBEE
:10232000204600F011FA2068016841F40041016084
:102330000020606284F8200010BD012010BD7047AD
:10234000406A704730B590F82040012C05D0022C2F
:1023500003D0416A41F480215DE00468002955D032
:102360002469A40754D04FF4D874056804EB011411
:102370002D5915F00405956005682D594ED0ED08CE
:10238000556005682C5904F00204D4604FF4DA74E7
:10239000056804EB01142D5905F00F05156105685A
:1023A0002D59C5F30725956105682C59240C5461F6
:1023B0004FF4DC72046802EB0112A4581C7004682C
:1023C000A458240A5C700468A458240C9C70046807
:1023D000A258120EDA704FF4DE72046802EB01129A
:1023E000A4581C710468A458240A5C710468A45899
:1023F000240C9C710468A258120EDA71006881B135
:10240000016941F020010161002030BDE468A8E7C6
:10241000416A41F400114162012030BD6D0D15602B
:10242000AFE7C16841F02001C160EDE72DE9F05F41
:102430000546006800244669D0F804908768D0F803
:102440000CB0D0F810A0D0F81880F10748D0F907E8
:1024500014D001218160B80703D5284600F0DFFAC7
:102460000CE0780702D54FF4006407E0380702D586
:102470004FF4805402E0284600F0D0FAF80516D553
:1024800029684FF480708860B80503D5284600F0AD
:10249000C8FA0CE0780502D544F4005407E038058A
:1024A00002D544F4804402E0284600F0B9FAF8036B
:1024B00016D529684FF480308860B80303D52846C4
:1024C00000F0B1FA0CE0780302D544F4004407E0D0
:1024D000380302D544F4803402E0284600F0A2FA22
:1024E000300707D55FEACB6004D52968102044F493
:1024F0000074C86070074FF0080707D55FEA0B70DB
:1025000004D52868C760284600F088F9B00706D5CA
:102510002868C068800702D0284600F081F970065C
:1025200007D55FEACA6004D52968102044F48064A6
:102530000861B00607D55FEA0A7004D5286807610C
:10254000284600F00BFAF00606D5286800698007D7
:1025500002D0284600F003FAB00308D55FEAC9604C
:1025600005D5296810204860284600F0F9F9F003E5
:1025700007D55FEA097004D528684760284600F04F
:1025800053FA300446D55FEA497040D5F00504D5CA
:102590005FEAC87001D044F00104B00504D55FEAD9
:1025A000887001D544F00204700504D55FEA4870D4
:1025B00001D544F00404300529D518F0700F26D059
:1025C00008F07000402815D006DC102809D020281B
:1025D0000AD0302816D10AE050280ED0602811D138
:1025E0000EE044F008040DE044F010040AE044F06A
:1025F000200407E044F0400404E044F0800401E0DB
:1026000044F480742868816921F07001816129682F
:1026100004204860002C05D0686A20436862284680
:10262000FFF78DFE00F000B830BCBDE8C09F70B56C
:10263000040003D094F8200010B104E0012070BD24
:10264000204600F0A1F82068016841F00101016016
:1026500000F0B4FD0546052604E000F0AFFD401B88
:102660000A2811D820684068C007F6D020680168A1
:1026700021F00201016000F0A1FD05460BE000F031
:102680009DFD401B0A2806D9606A40F40030606254
:1026900084F82060D2E7206840688007EFD4207E6D
:1026A0000128206801683DD021F080010160607E32
:1026B00001282068016838D021F040010160A07E27
:1026C00001282068016833D021F020010160E07EFC
:1026D0000128206801682ED041F010010160207FA0
:1026E00001282068016829D021F008010160607F7D
:1026F00001282068016824D021F004010160D4E998
:1027000002010843D4E90412114308436168491ED9
:1027100008432168C86100206062012084F820001D
:10272000002070BD41F08001C0E741F04001C5E7E5
:1027300041F02001CAE721F01001CFE741F0080184
:10274000D4E741F00401D9E710B500680C4988428C
:1027500015D10C48816D21F0007181654FF4C05195
:102760004FF0904000F098FB132001F033F8142054
:1027700001F030F8BDE81040162001F02BB810BD74
:10278000006400400010024010B586B004461421D9
:102790006846FDF7D4FD1F492068884237D11E489E
:1027A000816D41F000718165816D01F000710591CD
:1027B000C16C41F00101C164C06C694600F00100C8
:1027C00005904FF4C050009002200190002002902C
:1027D0000320039009200490C00600F0FFFB0022B4
:1027E0000521132001F014F8132001F004F8002251
:1027F0000521142001F00CF8142000F0FCFF002249
:102800000521162001F004F8162000F0F4FF06B0B0
:1028100010BD00000064004000100240704700003E
:1028200070B58CB002AB04AA00213548FFF78AFDD1
:1028300040B13348FFF784FD014632A004F0D6FCD6
:102840000CB070BD0598FF24384DB0F5801F03D043
:10285000B0F5881F25D027E00698042824D134A09D
:10286000059904F0C3FC9DF8090098B19DF8081083
:10287000FF2902D02A799142E2D1A88004F080F8A1
:102880002A4800940194FF23AA880121001DFEF725
:102890005DFAD5E7254AFF23921D0094002101949B
:1028A00029E00698042803D027A004F09FFCC7E77E
:1028B0001FA0059904F09AFC9DF80860002EE9D04D
:1028C0009DF809100029E5D09DF80A20002AE1D0E2
:1028D0009DF80B30002BDDD01448801D0670417030
:1028E0008270C370304604F083F8104AFF23921DB3
:1028F000009404210194A888FEF7C6F9A0E700001F
:10290000106A002043414E20726563656976652038
:102910006661696C6564214572726F7220636F64D1
:10292000653A2030782530386C580A0010000020B5
:1029300043414E49442072656365697665643A2077
:102940003078253038580A0043414E4944206D699B
:10295000736D617463686564210A00007047704795
:102960007047000070B5044690F82000012804D09C
:10297000606A40F40020606218E0022084F82000C1
:102980002068016821F00101016000F017FC054694
:102990000EE000BF00F012FC401B0A2808D9606A54
:1029A00040F400306062052084F82000012070BDF2
:1029B00020684068C007EDD1606270BD70B5044604
:1029C00090F82000022804D0606A40F48010606211
:1029D00014E02068016841F00101016000F0EEFBA5
:1029E00005460DE000F0EAFB401B0A2808D9606AA2
:1029F00040F400306062052084F82000012070BDA2
:102A000020684068C007EDD02068016821F002010D
:102A10000160012084F82000002070BD70477047DD
:102A20007047704770477047704710B590F8251091
:102A30000022022905D00421C16380F8242001204E
:102A400010BD01680B6823F00E030B6001680B6872
:102A500023F001030B6090F84410046C01F01C0398
:102A6000012101FA03F3636080F8251080F8242027
:102A7000104610BD10B590F825100024022903D08F
:102A80000421C16301241AE001680A6822F00E02E1
:102A90000A6001680A6822F001020A6090F8441096
:102AA000036C01F01C02012101FA02F25A6080F865
:102AB0002510002180F82410816B01B18847204641
:102AC00010BDF0B4016C0C6801680D6890F84420EA
:102AD00002F01C06042202FA06F3234211D06B070F
:102AE0000FD50B689B0603D40B6823F004030B601F
:102AF00090F8441001F01C018A40016C4A60016B9F
:102B00001DE0022303FA06F727424FF0000C4FF0B6
:102B1000010218D0AF0716D50C68A40605D40C68BE
:102B200024F00A040C6080F8252090F8441001F08D
:102B30001C018B40016C4B6080F824C0C16A0029E5
:102B40001AD0F0BC08470823B340234214D02B0707
:102B500012D50B6823F00E030B6090F84410036C41
:102B600001F01C0102FA01F15960C26380F82520CE
:102B700080F824C0416BE2E7F0BC704770B568B1E3
:102B80002B4C036814212B4AA34209D22A4C1C4423
:102B9000B4FBF1F18900C0E910210BE0012070BD08
:102BA000234C64421C44B4FBF1F189004164204988
:102BB00008390164022180F825101C6847F6F0717D
:102BC0008C43D0E902152943D0E904563543294303
:102BD00085692943C5692943056A29432143196049
:102BE0008168B1F5804F19D0036C0F21934202D157
:102BF00052F8A83F02E00E4AA032136890F8444011
:102C000004F01C04A1408B43136090F844304168E9
:102C100003F01C0399401368194311600021C1633C
:102C2000012280F8252080F82410084670BD00009D
:102C30000804024000000240F8FFFDBF70B50446E2
:102C400090F82400002501280CD0012084F82400ED
:102C500094F825600020012E06D084F82400022577
:102C6000284670BD022070BD022684F82560E0630E
:102C70002068066826F0010606602046FEF786F901
:102C8000206B00282068016802D041F00E0106E0A8
:102C900021F0040101602068016841F00A0101602F
:102CA0002068016841F001010160D9E770B5044670
:102CB00000F084FA0546601C02D004480078044401
:102CC00000F07CFA401BA042FAD370BD5C000020EB
:102CD0002DE9F05F054632488946017801290CD07C
:102CE0000126804606704CF2503B5846FFF7E2F84A
:102CF00007004FF0000A03D04EE0022000F054B865
:102D000051464046C8F804A0264C226892050AD5D0
:102D10002168490505D5216821F4806121600321DE
:102D200009E0067708E02268520504D5216821F4FD
:102D300080612160022101772868012807D04FF0C7
:102D4000FF31C9F8001040F2FA3BAE681DE0686838
:102D5000FFF76AF85846FFF7ADF80746606920F0BC
:102D60000400606116E030466968FFF76BF84CF2CA
:102D70005030FFF79FF80700606920EA0B006061A0
:102D800002D0C9F8006005E0761CD5E902010844CC
:102D9000B042E8D8FFF71AF888F800A03846ADE747
:102DA000680000200020024030BCBDE8C09F000049
:102DB0000348416941F00041416100207047000033
:102DC000002002402DE9FF5F254C06469046207802
:102DD0009A4601280BD0012020704CF2503B5846F7
:102DE000FFF768F807004FF0000904D02AE002203E
:102DF00004B000F039B84846C4F80490194D296869
:102E0000490504D5286820F48060286002202077D6
:102E100026B1012E09D0022E07D00CE042465346BF
:102E20000198FFF723F8012612E041460198FFF7C9
:102E30002BF8022E0AD05846FFF73CF84FEA00075D
:102E4000FEF7C4FF84F800903846D1E74FF480269F
:102E50005846FFF72FF807466869B0436861EFE707
:102E6000680000200020024030BCBDE8C09F000088
:102E7000064900204A69002A07DA054A8A60054A9D
:102E80008A604969002900DA012070470020024069
:102E900023016745AB89EFCD2DE9F84F00230126CB
:102EA000DFF818C10F2782E006FA03F414EA0102E2
:102EB0007CD023F003056544AA46D5F808909D0709
:102EC0004FEA157E07FA0EF505EA090B0095B0F1F9
:102ED000904F05D03A4DA84205D14FF0010816E0B9
:102EE0004FF0000813E0374DA84202D14FF002081E
:102EF0000DE0354DA84202D14FF0030807E0334DF5
:102F0000A84202D14FF0040801E04FF0070808FA88
:102F10000EF8D84526D1DFF8B880D8F8009029EA15
:102F20000209C8F8009008F10408D8F8009029EACE
:102F30000209C8F80090DFF8988008F10C08D8F86A
:102F4000009029EA0209C8F80090A8F10408D8F80E
:102F500000509543C8F80050009DDAF80820AA43B5
:102F6000CAF80820D0F800804FEA4309032202FA89
:102F700009F248EA0208C0F80080DD0800EB850588
:102F8000AA46D5F820804FEA43794FEAD96907FA73
:102F900009F528EA0508CAF8208085689543856008
:102FA0004568A5434560C4689443C4605B1C31FA1E
:102FB00003F27FF479AF00F00DB80000000001408B
:102FC0000004004800080048000C004800100048B9
:102FD0000004014018BCBDE8E08F00002DE9F04F6F
:102FE000DFF8AC9100230325A9F1040B85B04FF065
:102FF000010C0F2709F1040AABF1040EBFE000BF7A
:103000000CFA03F6324075D00C7904F00304012C5D
:1030100001D0022C1BD1846800945C0005FA04F8EE
:103020000494009C24EA08040094D1F80C80049CC9
:1030300008FA04F8009C48EA0408C0F808804468CC
:10304000B4430E79C6F300169E40264346600C79C1
:10305000E443A4070AD0C4684FEA430805FA08F617
:10306000B4438E6806FA08F62643C6600C7904F06D
:103070000304022C10D1DC0800EB84040294246ABF
:103080005E074FEAD66807FA08F6B4430E6906FAF7
:1030900008F62643029C266204684FEA430805FAB4
:1030A00008F6B4430E7906F0030606FA08F626433E
:1030B00006604C6814F4403F60D0364C266E46F0F3
:1030C00001062666246E23F0030604F00104009432
:1030D000314C34440294A4689E074FEA167807FAEC
:1030E00008F6B443B0F1904F05D02C4EB04204D155
:1030F000012612E042E000260FE0294EB04201D145
:1031000002260AE0274EB04201D1032605E0264EF2
:10311000B04201D1042600E0072606FA08F626434D
:10312000029CA660D9F800604C46D1F80480964312
:103130005FEAC82800D516432660DAF800405646F4
:10314000D1F8048094435FEA882800D514433460A2
:10315000DBF800405E46D1F8048094435FEA88388B
:1031600000D514433460DEF800407646D1F8048080
:1031700094435FEAC83800D5144334605B1C0A6886
:1031800032FA03F47FF43CAF05B000F00FB8000052
:103190000804014000100240000001400004004803
:1031A00000080048000C00480010004830BCBDE892
:1031B000C08F0AB1816170478162704701488068A1
:1031C000704700005C00002090F84120202A24D1A4
:1031D00090F84020012A20D0012280F840202422AB
:1031E00080F841200268136823F00103136002682D
:1031F000136823F480531360026813680B43136051
:1032000001680A6842F001020A60202180F841103A
:10321000002180F84010084670470220704790F85F
:103220004120202A22D190F84020012A1ED00122DC
:1032300080F84020242280F841200268136823F09F
:10324000010313600268136823F4706343EA0121E9
:10325000116001680A6842F001020A60202180F8CA
:103260004110002180F84010084670470220704746
:1032700070B5040004D094F84100002510B106E0B8
:10328000012070BD84F84050204600F0B3F924209E
:1032900084F841002068016821F001010160606844
:1032A000216820F0706008612068816821F4004185
:1032B0008160E0680128A06807D040F404402168DC
:1032C0008860E068022803D006E040F40040F6E79A
:1032D00021684FF40060486020684168114A11433A
:1032E00041602068C16821F40041C160D4E9040153
:1032F0000843A16940EA01202168C860D4E90701B8
:103300000843216808602068016841F001010160FC
:103310006564202084F84100256384F84250002031
:1033200070BD0000008000022DE9FF4F83B004460D
:10333000DDE9108790F84100DDF848909A46934601
:10334000202874D15FEA080014D09FB194F840009F
:1033500001286CD0012084F84000FFF72FFF0646BB
:10336000012200901923D103204601F029FF0028F3
:1033700071D103E04FF4007060646CE0222084F8A7
:103380004100402084F8420000256564C4F8248090
:1033900067856563CDE9009653465A4620460499F1
:1033A00001F092FE10B184F8405054E0618D354830
:1033B000FF274FF080784FF0007AFF2904D9278546
:1033C0003A464346009005E0618D2185009094F8CF
:1033D000282053462046049901F0DAFE4B4600228D
:1033E00004212046009601F0EBFEA0BB2068406A55
:1033F000616A0870606A401C6062208D401E81B264
:103400002185608D401E6085608DD8B1D1B94B4655
:10341000002280212046009601F0D2FED8B9608DAE
:10342000FF2805D927853A464346009506E026E061
:10343000608D2085009594F82820534620460499F5
:1034400001F0A6FE608D0028C8D1324649462046CC
:1034500001F0E2FE18B1012007B000F017B82168B2
:103460002020C86121684A68074B1A404A6084F8E6
:10347000410084F8425084F840500020ECE70220DC
:10348000EAE700000024008000E800FE30BCBDE850
:10349000C08F00002DE9FF4F83B00446DDE910879F
:1034A00090F84100DDF848909A469346202871D163
:1034B0005FEA080014D09FB194F84000012869D059
:1034C000012084F84000FFF779FE064601220090B3
:1034D0001923D103204601F073FE00286ED103E0CA
:1034E0004FF40070606469E0212084F841004020BE
:1034F00084F8420000256564C4F82480678565630C
:10350000CDE9009653465A462046049901F00EFE36
:1035100010B184F8405051E0608DFF274FF0807863
:103520004FF0007AFF2804D927853A464346009594
:1035300005E0608D2085009594F8282053462046AC
:10354000049901F025FE32464946204601F08AFEE4
:10355000A0BB606A216800788862606A401C606273
:10356000608D401E6085208D401E80B22085618D5B
:10357000D9B1D0B94B46002280212046009601F0F7
:103580001FFED8B9608DFF2805D927853A464346E6
:10359000009506E026E0608D2085009594F82820AF
:1035A00053462046049901F0F3FD608D0028CAD1EE
:1035B00032464946204601F02FFE18B1012007B0DF
:1035C00000F014B820682021C16120684268064BD1
:1035D0001A40426084F8411084F8425084F8405008
:1035E0000020ECE70220EAE700E800FE30BCBDE87E
:1035F000C08F00002DE9F0419EB00646142117A8A7
:10360000FCF79DFE5C216846FCF799FE2E49306868
:10361000884255D14020002400900C94684600F068
:1036200089F908B1FDF70CFD284DE86C40F0010068
:10363000E864E86C17A900F001001C904FF4C0602A
:1036400017901220CDE918040420CDE91A404FF05C
:103650009040FFF7C3FCA86D40F40010A865A86D6A
:103660001C4D00F400101C90194828600527C5E97E
:1036700001744FF08008C5E903486C61AC61EC61EE
:1036800028462C62FFF77AFA08B1FDF7D9FCF563FA
:10369000AE62104D0E4848351430E5E802071020A0
:1036A000A5E811010B4845F814494830AC61EC61BC
:1036B0002C62FFF763FA08B1FDF7C2FCB563AE6296
:1036C0001EB0BDE8F0810000005400400010024030
:1036D0006C0402408C6A0020024881680278114420
:1036E000816070475C00002010B50024032000F0CA
:1036F000AFF80F2000F008F808B1012401E000F055
:103700004FF8204610BD000030B505461F4887B071
:10371000816D41F010018165806D06A900F01000F7
:10372000009001A800F006FB0498B0B100F022FB65
:1037300040001749174AB0FBF1F11748491E0260D3
:10374000416040F2E7320021C0E9032181608161DC
:1037500001F068F8040003D015E000F00BFBE8E787
:103760000D4801F091F804000DD1362000F043F827
:10377000102D07D200222946362000F049F80748CC
:10378000056000E0012407B0204630BD0010024073
:1037900040420F0000100040546C002060000020E8
:1037A0000B4882B0016E41F001010166016E01F02B
:1037B00001010091816D41F080518165806D002291
:1037C00000F0805000900F21901E02B000F020B851
:1037D0000010024000280DDB00F01F020121914083
:1037E0004009800000F1E020C0F88011BFF34F8F46
:1037F000BFF36F8F7047002809DB00F01F02012123
:1038000091404009800000F1E020C0F800117047AD
:10381000F0B40E4B1B680C46C3F30223C3F107053B
:10382000042D00D90425191D072901D2002300E029
:10383000DB1E012606FA05F1491E214099409E40F3
:10384000761E16403143F0BC03F00CBD0CED00E0D9
:10385000064900F0070208684FF6FF03184040EAE7
:103860000220034A10430860704700000CED00E09E
:103870000000FA051649B0F5007F0868C0F3412042
:1038800009D0022805D0086820F4C06040F48060A8
:103890000860002070470128FBD0086820F4C06051
:1038A00040F4007008600B483222006850430A4A16
:1038B000B0FBF2F0401C00E0401E4A69520501D501
:1038C0000028F9D148694005E3D50320704700007E
:1038D000007000408800002040420F000B490A6839
:1038E00022F00702921C0A6009490A6842F00402A9
:1038F0000A60012807D040BF20BF20BF086820F021
:1039000004000860704730BFF8E700000070004016
:1039100010ED00E00248006800F4C060704700004D
:10392000007000400248016841F4807101607047F6
:10393000007000402DE9F84F044600270088A84D8C
:103940003E46000515D5606C60B1B0F5000F04D09F
:10395000B0F5400F2BD001270AE0E86840F4803032
:10396000E86024E00021201D02F068FE07001ED060
:103970003E46206880033AD5A86D4FF00008C0008D
:1039800009D4A86D40F08050A865A86D4FF00108DB
:1039900000F080500090DFF84CA2DAF8001041F4FB
:1039A0008071CAF80010FFF709FC814610E0D5F8D5
:1039B0008800616C20F440000843C5F88800D8E70F
:1039C000FFF7FCFBA0EB0900022801D9032705E063
:1039D000DAF80000C005F3D5002F7DD04FEA0706C6
:1039E000B8F1000F03D0A86D20F08050A8652078B2
:1039F000C00707D0D5F88800216A20F003000843EB
:103A0000C5F888002078800707D5D5F88800616A56
:103A100020F00C000843C5F888002078400707D53F
:103A2000D5F88800A16A20F030000843C5F8880066
:103A30002078800607D5D5F88800E16A20F4406038
:103A40000843C5F888002088800507D5D5F8880088
:103A5000E16B20F440200843C5F888002088400529
:103A600007D5D5F88800216C20F440100843C5F82C
:103A700088002078400607D5D5F88800216B20F40F
:103A800040500843C5F888002078000607D5D5F8CF
:103A90008800616B20F440400843C5F88800208806
:103AA000C00507D5D5F88800A16B20F44030084345
:103AB000C5F8880020684FF0006700034FF0806869
:103AC00050D5D5F88800A16C20F040600843C5F8B7
:103AD0008800A06CB84200E005E03BD1E86840F403
:103AE0008010E8603EE0D5F8900010F4407014D0EB
:103AF000A16D814211D0D5F89000D5F8901020F436
:103B0000407041F48031C5F89010D5F8901021F440
:103B10008031C5F89010C5F89000C00711D0FFF7AC
:103B20004DFB074641F2883907E000BFFFF746FB2F
:103B3000C11B494501D9032652E7D5F890008007FB
:103B4000F4D5D5F89000A16D20F440700843C5F875
:103B5000900045E7404505D10121201D02F06EFD92
:103B600000B106462068400317D5D5F88800E16CFF
:103B700020F040600843C5F88800E06CB84204D1EA
:103B8000E86840F48010E86007E0404505D1012175
:103B9000201D02F053FD00B106462088400411D5D7
:103BA000D5F88800216D20F040500843C5F8880002
:103BB000206DB0F1805F05D10221201D02F03EFD95
:103BC00000B106462088000406D555F8880F616DBF
:103BD00020F0804008432860304600F005B800001F
:103BE000001002400070004018BCBDE8E08F0000EB
:103BF0002DE9F0470F4605006BD0494E306800F0C4
:103C00000700B84209D2306820F00700384330601E
:103C1000306800F00700B8425BD12878414C80073B
:103C20000AD5A868A16801F0F001884204D9A1680A
:103C300021F0F0010143A1602878C0072CD068680A
:103C4000032811D0022812D0216898B14905002913
:103C50003FDAA16821F003010143A160FFF7AEFA4A
:103C6000804641F2883910E021688901EFE7216838
:103C70008903ECE78907EAE7FFF7A0FAA0EB080160
:103C8000494502D90320BDE8F087A068696800F0C3
:103C90000C00B0EB810FEFD1287880070AD5A86817
:103CA000A16801F0F001884204D2A16821F0F0017E
:103CB0000143A160306800F00700B8420BD93068BA
:103CC00020F0070038433060306800F00700B84249
:103CD00001D00120D7E72878400705D5A068E9681A
:103CE00020F4E0600843A0602878000706D5A068AB
:103CF000296920F4605040EAC100A06000F05EF83D
:103D0000A168094AC1F30311515C01F01F01C840C9
:103D10000649086006480068BDE8F047FFF7F4BCB4
:103D20000020024000100240E0A7000888000020A8
:103D3000600000200F2202600C4A936803F0030326
:103D40004360936803F0F0038360936803F4E063D7
:103D5000C36092684FF4E06303EAD2020261044850
:103D6000006800F007000860704700000010024083
:103D7000002002400548064900688968054AC1F3E9
:103D80000221515C01F01F01C840704788000020EB
:103D90000010024020A8000805480649006889680C
:103DA000054AC1F3C221515C01F01F01C8407047B0
:103DB000880000200010024020A8000870B52549A6
:103DC000002318468A68CC6812F00C0204F003063F
:103DD000214C4FEA640509D00C2A05D0042A32D0C0
:103DE000082A00D1284670BD012E10D10B681B0790
:103DF00004D4D1F89430C3F3032302E00B68C3F377
:103E00000313164E56F82330DAB10C2AEBD1C868EA
:103E100000F00300022818D0032818D01846CA68FA
:103E2000CB68C2F30212C3F306234343521CB3FB15
:103E3000F2F2C868C0F34160401C4000B2FBF0F0F1
:103E400070BD184670BD204670BD2046E7E7284685
:103E5000E5E70000001002400024F400F0A700088D
:103E60002DE9F84304006FD0FA4DA86800F00C0665
:103E7000E86800F003072078C00664D576B10C2E00
:103E800001D1012F0AD0A069002828687AD040F01B
:103E900001002860FFF792F980465DE028688007FE
:103EA00002D5A0690028DED0216A2868000703D562
:103EB000286800F0F00004E0D5F89400F02202EA4F
:103EC0001010814216D9084602F04EFC00283BD162
:103ED000286840F0080028602868216A20F0F00077
:103EE000084328606868E16920F47F4040EA0120C7
:103EF000686016E0286840F0080028602868216A99
:103F000020F0F000084328606868E16920F47F40F1
:103F100040EA0120686026B9206A02F025FC0028EA
:103F2000D5D1FFF74BFFA968CB4AC1F30311515C10
:103F300001F01F01C840C9490860C9480068FFF77F
:103F4000E3FB00287ED12EE0CAE000BFFFF736F980
:103F5000A0EB0800022876D828688007F6D52868E4
:103F600040F0080028602868216A20F0F00008432B
:103F700028606868E16920F47F4040EA01206860B9
:103F800011E0FFE720F001002860FFF717F98046F5
:103F900006E000BFFFF712F9A0EB08000228DAD80C
:103FA00028688007F6D42078C00740D0082E18D0A3
:103FB0000C2E01D1032F14D06068B0F5803F17D0CC
:103FC000B0F5A02F286817D020F48030286028682A
:103FD00020F4802028606068E0B1FFF7EFF88046A9
:103FE00014E02868800322D56068002878D01EE09D
:103FF000286840F48030EDE740F480202860F7E73F
:10400000FFF7DCF8A0EB08006428A4D82868800338
:10401000F6D50CE0FFF7D2F8804605E0FFF7CEF8C2
:10402000A0EB0800642896D828688003F6D420788E
:1040300080073BD5042E11D00C2E01D1022F0DD0BC
:10404000E06801E0AAE1FFE0002828681ED040F403
:1040500080702860FFF7B2F807460CE0286840053A
:104060000CD5E0680028C1D008E000BFFFF7A6F833
:10407000C01B022893D828684005F7D56868217CC2
:1040800020F0F85040EA016068600FE020F4807092
:104090002860FFF793F8074605E000BFFFF78EF8AA
:1040A000C01B0228B1D828684005F7D42078000743
:1040B00029D560690028D5F8940012D040F001009D
:1040C000C5F89400FFF77AF8074604E0FFF776F8A2
:1040D000C01B022899D8D5F894008007F6D512E0C5
:1040E0002BE120F00100C5F89400FFF767F80746C0
:1040F00005E000BFFFF762F8C01B022885D8D5F89D
:1041000094008007F6D42078400766D5A86D002774
:10411000C00008D4A86D40F08050A865A86D0127A4
:1041200000F0805000904F480168C90512D4016822
:10413000814641F480710160FFF740F8804605E058
:10414000FFF73CF8A0EB080002287DD8D9F8000062
:10415000C005F5D5A068012816D00528D5F890002F
:1041600017D020F00100C5F89000D5F8900020F09D
:10417000040000BFC5F89000A06841F28839C0B1C2
:10418000FFF71CF880460FE0D5F8900040F00100E2
:10419000F0E740F00400C5F89000F5E7FFF70EF8EF
:1041A000A0EB080149454FD8D5F890008007F5D518
:1041B0000EE0FFF703F8804606E000BFFEF7FEFFC3
:1041C000A0EB080149453FD8D5F890008007F5D409
:1041D0001FB1A86D20F08050A8652078800628D5F2
:1041E000606A0028D5F8980012D040F00100C5F8A8
:1041F0009800FEF7E3FF074605E000BFFEF7DEFF8D
:10420000C01B022820D8D5F898008007F6D510E00A
:1042100020F00100C5F89800FEF7D0FF074604E043
:10422000FEF7CCFFC01B02280ED8D5F898008007F7
:10423000F6D4A06AF0B3022816D00C2E7DD02868E0
:1042400020F08070286000E0A7E0FEF7B7FF04468A
:10425000A6E0000000100240E0A70008880000204F
:104260006000002000700040E868E26A00F003018E
:10427000914228D1216B00F070020901103991425E
:1042800021D1626B00F4FE41B1EB022F1BD194F8F7
:10429000382000F07841B1EBC26F14D1A18F00F447
:1042A000C00249084905A1F5001191420BD194F8CB
:1042B000401000E06AE04908490600F0C060A1F142
:1042C000007181424BD00C2E73D02868400170D40D
:1042D000286820F080702860FEF770FF064604E032
:1042E000FEF76CFF801B022857D828688001F7D49E
:1042F000F4E90B016FF00F0202EB01110843218A70
:104300005204490802EB4151A26841EA02210843E4
:10431000217D4FF07E42490802EB41610843217B39
:1043200040EAC160E968244A11400843E86028680F
:1043300040F080702860E86800E03AE040F080706B
:10434000E860FEF73BFF044605E000BFFEF736FFDE
:10435000001B022821D828688001F7D527E02868AB
:10436000800124D4286840F080702860E86840F01C
:104370008070E860FEF722FF044604E0FEF71EFFAF
:10438000001B022809D828688001F7D50FE000BF7C
:10439000FEF714FF001B022802D90320BDE8F883B2
:1043A00028688001F4D4E86804490840E8600020E7
:1043B000F4E70120F2E700008C809D01FCFFEEFE97
:1043C0002DE9F047044690F8200001281ED0012670
:1043D00084F82060022084F821002168CA20486205
:1043E0002168532048622068816821F480618160DF
:1043F0002068816821F480418160FEF7DFFE054678
:1044000000274FF0FF084FF47A7911E00220BDE851
:10441000F08700BFFEF7D2FE401B484508D921684F
:10442000C1F82480032084F8210084F82070EEE78E
:104430002068C0684007EDD52168C1F8248084F861
:10444000216084F820700020E1E700002DE9F05F92
:10445000044690F8200093468A46012825D001267C
:1044600084F82060022084F821002168CA20486274
:104470002168532048622068816821F4806181604E
:104480002068C16801F0800161F49061C16020681A
:10449000C0684FF0000740064FF0FF081AD4FEF73F
:1044A0008DFE05464FF47A7910E0022000F03CB80A
:1044B000FEF784FE401B484508D92168C1F82480D6
:1044C000032084F8210084F82070EFE72068C0689A
:1044D0004007EDD52168C1F814A02068816821F05B
:1044E000070141EA0B0181600E48016841F4801127
:1044F00001600C480830016841F4801101602068B7
:10450000816841F4804181602068816841F4806164
:1045100081602168C1F8248084F8216084F82070CB
:104520000020C3E70004014030BCBDE8C09F00008C
:1045300005A002F05BFE012004F072FA4FF4007057
:10454000FFF798F902F09EFE5254432063616C6CB1
:104550006261636B0A00000010B50B4904464FF41A
:10456000801008602068C168490508D5C16801F05D
:10457000800161F49061C1602046FFF7D9FF0120FE
:1045800084F8210010BD00001404014010B504009F
:104590004FF0010044D094F8210028B9002084F89D
:1045A0002000204600F040F8022084F82100216815
:1045B000CA204862216853204862204602F01EF952
:1045C00000282DD120688168164A11408160216839
:1045D00088686268A369104322691A43104388609F
:1045E0002168E068086120680169228941EA024186
:1045F0000161204602F026F9002811D12168CA6C19
:1046000022F00302CA646269E16911432268D36C33
:104610001943D1642268FF215162012184F82110DD
:1046200010BD0000BFFF8FFF10B598B004465C219D
:104630006846FBF784FE0F492068884218D14FF482
:1046400000300090401216906846FFF773F908B1E9
:10465000FCF7F6FC084850F8901F41F40041016057
:10466000002205210320FFF7D3F80320FFF7C3F84A
:1046700018B010BD002800400010024070B504467C
:1046800090F820000B4601281BD0012684F82060FA
:10469000022084F82100B2B19878D97840EA014527
:1046A00058781978000240EA413005432168CA2051
:1046B0004862216853204862204602F09FF8D0B13A
:1046C00020E0022070BD5878C10603D500F0EF004D
:1046D0000A305870D87802F085F80504587802F04E
:1046E00081F845EA0025987802F07CF805431878AF
:1046F00045EA4035DAE7084805402068456020462D
:1047000002F0A0F82268FF21516208B984F8216004
:10471000002184F8201070BD3FFFFF002DE9F0411B
:10472000044690F8200090460D46012811D001273C
:1047300084F82070022084F821002168CA20486291
:10474000216853204862204602F058F8002618B12C
:1047500029E00220BDE8F0812068B8F1000F8068F0
:104760004FEA406024D0002800DBEE70A87829785A
:10477000EA7840EA01406978090241EA8251084337
:1047800018490840216808602068816821F4802168
:104790008160D5E90301084321688A681043886075
:1047A000204602F04FF82268FF215162A0B115E0C7
:1047B000002800DBEE70287802F014F80304687813
:1047C00002F010F843EA0023A87802F00BF8034344
:1047D000E87843EA8050D3E784F8217084F82060B9
:1047E000B8E700007F7F7F0070B504460068C168AD
:1047F00021F0A001C160FEF7E1FC05464FF47A7696
:1048000007E000BFFEF7DAFC401BB04201D90320ED
:1048100070BD2068C0688006F4D5002070BD704768
:104820007047704710B5040003D094F83D0010B1F4
:1048300007E0012010BD002084F83C00204600F075
:1048400022F8022084F83D00211D206802F086F93C
:10485000012084F8480084F83E0084F83F0084F882
:10486000400084F8410084F8420084F8430084F852
:10487000440084F8450084F8460084F8470084F832
:104880003D00002010BD704790F83D10012901D077
:1048900001207047022180F83D100168CA6842F08B
:1048A0000102CA6000680B49884205D0B0F1804F10
:1048B00002D00949884207D18168084A1140062977
:1048C00006D0B1F5803F03D0016841F001010160DD
:1048D00000207047002C014000400140070001000B
:1048E000704770B50446006801694FF00005C94380
:1048F000890715D4C168C943890711D4E91E01612C
:1049000001202077206880698007204602D0FFF7C9
:10491000E7FF04E000F0A7F8204600F0A5F82577AF
:1049200020680169C943490717D4C168C9434907C9
:1049300013D46FF0040101610220207720688069A0
:1049400010F4407F204602D0FFF7CAFF04E000F0D9
:104950008AF8204600F088F8257720680169C94365
:10496000090716D4C168C943090712D46FF00801BA
:104970000161042020772068C0698007204602D0AA
:10498000FFF7AEFF04E000F06EF8204600F06CF890
:10499000257720680169C943C90617D4C168C9438E
:1049A000C90613D46FF01001016108202077206838
:1049B000C06910F4407F204602D0FFF791FF04E069
:1049C00000F051F8204600F04FF825772068016983
:1049D000C943C90708D1C168C943C90704D1891EA1
:1049E0000161204600F042F820680169C9430906C8
:1049F00009D4C168C943090605D46FF0800101617B
:104A00002046FFF70DFF20680169C943C90509D495
:104A1000C168C943090605D46FF48071016120465D
:104A2000FFF7FDFE20680169C943490609D4C16842
:104A3000C943490605D46FF040010161204600F0EA
:104A40001FF820680169C94389060BD4C168C943AE
:104A5000890607D46FF0200101612046BDE870404F
:104A6000FFF7DFBE70BD7047704700000068034964
:104A7000884201D1FEF730BE7047000000100040B0
:104A800070477047704770472DE9F041026804464F
:104A9000D0691168936840F60F0528424FF0000571
:104AA00005D186067ED58E067CD5616E1BE1994FB9
:104AB00003F001060F40374374D0C70709D0CF0574
:104AC00007D501271762D4F8802042F00102C4F80C
:104AD000802082070AD5DA0708D0276802223A62C6
:104AE000D4F8802042F00402C4F8802042070AD59E
:104AF000DA0708D0236804221A62D4F8802042F032
:104B00000202C4F8802002070CD501F020023243D3
:104B100008D0236808221A62D4F8802042F00802E4
:104B2000C4F8802002050BD54A0109D523684FF44B
:104B300000621A62D4F8802042F02002C4F880207B
:104B4000D4F88020002A35D0800605D5880603D504
:104B5000616E09B120468847D4F8800021688968D1
:104B6000490602D410F0280F26D0204602F03CF966
:104B70002068806840061AD52068083050E8001F79
:104B800021F0400140E80012002AF5D1206F70B1F9
:104B900061498163206FFDF76DFF00280AD0206F07
:104BA000816B01E00EE02046BDE8F0410847204659
:104BB000FFF769FFBDE8F0812046FFF764FFC4F806
:104BC0008050F7E7276E2026012F7BD1C70679D5C5
:104BD000CF0677D51020106220688068400641D546
:104BE000216F086840680004000CE3D0B4F8582036
:104BF0008242DFD9A4F85A000868006880062AD4E7
:104C0000206850E8001F21F4807140E80012002A5B
:104C1000F6D12068083050E8001F21F0010140E87B
:104C20000012002AF5D12068083050E8001F21F05A
:104C3000400140E80012002AF5D1E66725662168A8
:104C400051E8000F20F0100041E80002002AF6D1E0
:104C5000206FFDF7EAFEB4F85800B4F85A10401A75
:104C600081B22AE0B4F85800B4F85A10401A81B260
:104C7000B4F85A0000289DD000299BD0226852E841
:104C8000000F20F4907042E80003002BF6D120685A
:104C9000083050E8002F22F0010240E80023002BEA
:104CA000F5D1E66725666566226852E8000F20F0B8
:104CB000100042E80003002BF6D12046FFF7E1FE8A
:104CC00078E7FFE7C70209D55B0207D54FF48010EC
:104CD00010622046BDE8F041FFF7D4BE020606D5BB
:104CE0000A0604D5A16E00297FF45DAF62E7400695
:104CF000E6D54806E4D52046026852E8001F21F0B8
:104D0000400142E80013002BF6D18667856600F06B
:104D10003AF94FE720010004ED6C000810B50400DB
:104D200002D0A06F10B107E0012010BD002084F870
:104D30007400204600F026F82420A067206801684F
:104D400021F001010160204602F080F80128ECD03A
:104D5000606A10B1204601F037FF2068416821F4F5
:104D6000904141602068816821F02A0181602068BB
:104D7000016841F0010101602046BDE8104001F0EA
:104D800087BF00002DE9F0439DB00646142117A807
:104D9000FBF7D5FA5C216846FBF7D1FA3249306857
:104DA00088425DD102270024684600970994FEF7E7
:104DB000C1FD08B1FCF744F92C48816D41F4003184
:104DC0008165816D01F400311C91C16C41F00101DC
:104DD000C164C06C17A900F001001C900C20CDE943
:104DE00017070320CDE9194007201B904FF0904092
:104DF000FEF7F4F81F4D1E484FF080092860C5E902
:104E00000174C5E903496C614FF40058AC61C5E910
:104E100007482846FDF7B2FE08B1FCF711F93567DF
:104E2000AE62144D124848351430E5E802071020F0
:104E3000A5E811020F4845F814494830AC61C5E9AE
:104E40000748FDF79BFE08B1FCF7FAF8F56600226B
:104E500005212620AE62FEF7DBFC2620FEF7CBFC08
:104E60001DB0BDE8F0830000004400400010024087
:104E70006C000240C46B002030B4C36F202B20D1E3
:104E8000E1B1DAB190F87430012B1AD0012380F827
:104E90007430002303660C4C0368A3420BD05B689C
:104EA0001B0208D5046854E8003F43F0806344E8DF
:104EB0000035002DF6D130BC02F0C8B8012030BC5E
:104EC00070470220FBE700000080004070477047F9
:104ED0002DE9F8430446806F1F4616460D462028EC
:104EE0004FD1CDB1C6B194F87400012849D001204A
:104EF00084F874004FF00008C4F880802120A06777
:104F0000FEF75CF9A4F850608146A4F85260A068EE
:104F1000B0F5805F03D004E00120BDE8F88320698C
:104F200028B12E465FF0000584F8748010E000265A
:104F3000FAE78021204602F0DBF8B8B9C6B116F8CE
:104F4000010B21680885B4F85200401EA4F85200F5
:104F5000B4F852004B464FF0000200970028E8D109
:104F60004FF04001204602F0C3F830B10320D4E7EF
:104F700035F8020BC0F30800E3E72020A06700200B
:104F8000CBE70220C9E77047FEE701688A69D24390
:104F9000920701D400228A6200688169C943C90767
:104FA00003D0816941F00101816170472DE9F0472B
:104FB0000446006888461746816900252E46C906C2
:104FC000A9464FF0200A47D51021C16137E000BF44
:104FD000B8F1FF3F33D0FEF7F1F8C11B414502D8CD
:104FE000B8F1000F2BD12068416894F8422001F4F9
:104FF00080418369DB431B041CD4B1F5804F19D079
:10500000202A17D0416841F480414160FEF7D6F86C
:1050100007460FE0FEF7D2F8C01B19280AD9606CCA
:1050200040F02000606484F841A084F8429084F845
:105030004090012520688069C0438006EAD420683A
:105040008069C0F340102843C2D015B92168C1F867
:105050001CA046F00406012521688869C20505D513
:105060004FF4807246F00106CA610125410509D559
:1050700022684FF4806146F00806D1610125800561
:1050800002D40AE0800507D521684FF4007046F08D
:105090000206C861012500E08DB12046FFF775FFCB
:1050A00054F8240B4168074A11404160206A30439C
:1050B000206284F81DA084F81E9084F81C90284675
:1050C000BDE8F08700E800FE2DE9F84304461646E7
:1050D000DDE9089714489846DAB20090002320468C
:1050E00000F056F83A464946204600F0BBF8B8B9F9
:1050F000F5B2B8F1010F08D02168300A88623A464B
:105100004946204600F0AEF850B9206885624B460B
:10511000002240212046009700F052F8002800D0DD
:105120000120BDE8F8830000002000802DE9F8434D
:105130000446164615489846DDE90897DAB2C302D8
:105140000090204600F024F83A464946204600F0F8
:1051500089F8B8B9F5B2B8F1010F08D02168300A62
:1051600088623A464946204600F07CF850B92068EB
:1051700085624B46002280212046009700F020F8EF
:10518000002800D00120BDE8F88300000020008046
:1051900010B5C1F3090141EA02410268029C1943BA
:1051A0002143506821F000414FF4806303EA5453D7
:1051B000024C234398430843506010BDFF63FF0334
:1051C0002DE9F0411D4617460E460446DDF81880CD
:1051D00008E0681C06D0FDF7F1FFA0EB0800A8422C
:1051E0000BD855B12068806936EA000012D0002043
:1051F000B842EED00020BDE8F08154F8440F40F0F2
:10520000200044F80409202060700020A070207065
:105210000120F0E70120EBE770B516460D46044685
:105220000DE0324629462046FFF7C0FE08B10120B6
:1052300070BDFDF7C3FF801BA84207D835B12068B9
:105240008069C0438006ECD4002070BD54F8440F40
:1052500040F0200044F80409202060700020A07075
:105260002070E4E770B516460D4604460FE032465E
:1052700029462046FFF79AFE08B1012070BD681C40
:1052800005D0FDF79BFF801BA84207D835B12068E9
:105290008069C0438007EAD4002070BD54F8440FF1
:1052A00040F0200044F80409202060700020A07025
:1052B0002070E2E710B5002201EB420303F5005332
:1052C000B3F87A4A844203D0B3F8703A834201D1EA
:1052D000012010BD521C052AEEDB002010BD2DE977
:1052E000FF479A4691460C460646002501F50068A0
:1052F000B6EE001A4FF6FF77C1E0C0F34712A0EBFD
:105300004211C9B2B9F1010F0DD0B9B301296CD066
:105310001E296AD01F2970D0801E80B25146FFF727
:10532000C9FF60B376E05AB3172A3BD049B304EB08
:1053300080001F2910ED210A4FD08DED000A36F8AC
:105340001500042104EB800010ED1F0A8DED010A09
:1053500036F8150004EB800090ED1F0A8DED020A6F
:1053600036F8150004EB800090ED210A68468DEDBB
:10537000030AFCF7B8FE36F8150010E030E041E013
:1053800000E023E031B11F2907D004EB800090ED4D
:105390001F0A1FE094ED210A01E094ED3E0A04EBA0
:1053A000800068E061B11F290DD004EB800010ED92
:1053B000210A50ED1F0A30EE200A20EE010A5AE0C1
:1053C00098EDC10AEBE798EDDE0AE8E704EB800010
:1053D00010ED1F0AD0ED210AEDE7D0ED1F0AEAE734
:1053E00004EB800090ED010A45E004EB800010ED35
:1053F000010AD0ED010ADEE7FFE704EB800010EDC3
:10540000010A38E036F815005146801C80B2FFF7DB
:1054100051FF10B136F81500E7E736F8150004EB38
:10542000800090ED010AD0ED020A30EE600A8DEDA9
:10543000000A36F8150004EB800050ED010A50ED2B
:10544000021A70EEE10AF0EEC01ACDED010AB0EEDC
:10545000E02A36F81500F4EEC21A04EB8000F1EEF3
:1054600010FA04DD10ED010A30EE200A03E0D0ED61
:10547000010A30EE800A6D1CEDB280ED000A36F8AC
:105480001500B8427FF439AF00F000B80FBCBDE89A
:10549000F08700002DE9F74F06462DED020B0D4673
:1054A0002DED108B88B0B0EE609AB0EE40EAB0F807
:1054B00082060290304600F089FBF0EE408A2946D1
:1054C000304600F017FBB0EE408A9FEDFE0A41F631
:1054D000506038EE001A39EE000A405D21EE011AE4
:1054E00020EE000A61EE010A20EE000A30EE601A9A
:1054F000C1EE0E0A30EE609AFBF7D7F841EC110BC3
:105500009FEDF1ABB0EE4A0AF0EE6A0A01F0CCFE74
:1055100051EC100BFBF7E9F805F500540DEE900A7D
:1055200094F8540AFBF7C1F841EC110BB0EE4A0AAB
:10553000F0EE6A0A01F0B8FE51EC100BFBF7D5F85B
:105540000DEE100A95F84C0CFBF7AFF841EC110B7F
:10555000B0EE4A0AF0EE6A0A01F0A6FE51EC100B1A
:10556000FBF7C3F8B7EE00FAD5ED0B0A9FEDD81A9A
:10557000B0EE4F0A0AEE900A00EE810AD54BCFEE4C
:10558000000ACDED030A8DED04FAB5F94400D5ED1E
:105590000C0A00EE100AB8EEC01AB0EE4F0A00EE88
:1055A000810A8DED050AB5F94610F0EE400A081A99
:1055B00000EE100AD5ED0D1AB8EEC01AB0EE4F0A83
:1055C00001EE810A20EE200A8DED060AB6F81406D7
:1055D00000EE100AB8EE400A10EE100ADFEDBE0A27
:1055E000984201DD30EE600AB5F91400802101EE29
:1055F000100AB6F880064FEA0D02B8EEC11A01EAA9
:105600005017B6F81006C1EE009A00EE100AB8EE78
:10561000400A8DED000AB6F8500600EE100A002090
:10562000B8EE400A8DED010A02EB8001994691ED3A
:10563000000A10EE10CA9C4505DDDFEDA70A30EE2A
:10564000600A81ED000A20EE290A401C022881ED43
:10565000000AE9DBB3EE090A95ED081A38EE40AA14
:10566000B4F9600AF0EE4F0A00EE100A41EE0A0AA1
:1056700095ED071AB8EEC00A60EE801A9FED970A02
:1056800005F5205A78EEC0EAB0EE4F0A01EE2E0A78
:105690009DED001A01EEC01A8DED001AB4F9620AF0
:1056A00095F8251001EE100AB942B8EEC11A02D1E0
:1056B00020EE811A05E0DAED991A31EE211A21EE79
:1056C000201ADDED010A002441EE400ACDED010A69
:1056D0009FED83CBE31704EB936104EBD360891157
:1056E0004011494200EB410042B204EBD47040103B
:1056F000404204EB400004F1020C50404FEAEC78C9
:105700004FFA80FB0CEB987CE01C4FEAE0784FEA04
:10571000AC0C00EB9870611CACEBA0004FEAE17C94
:1057200001EB9C7100EBA10004EB9371A0EBA100D5
:105730005342012101EB4301484341B2002F7DD088
:105740004FEA0B00B6F88236834278D136F814005F
:1057500000EE100AB8EE400A10EE100A484503DDCC
:10576000DFED5D0A30EE600A05EB840000F5805342
:1057700093ED941A00F5E05320EE290AC1EE2D0AAC
:10578000D3ED951A05EB4403B3F94E3C81EE8D1A27
:1057900001EE903A95F82530B8EEE12AF0EE4F1A76
:1057A000BB4240EE8A1AF0EE4F0A62EE211A41EE39
:1057B0002E0A01EEE00A13D04FF0FF3303EB420252
:1057C00000EE902A9AED9B1AF8EEE00A01EE200A0C
:1057D00000EE901A9AED9A1AF8EEE00A01EE600ACD
:1057E000029A694601EB8201D5ED060A91ED001A95
:1057F00000EEC10A90ED131A286BC0EE0E8A9FEDE1
:105800003A0A6AEE800A80EE810A95ED0A1AF0EEF5
:105810004F0A41EE0A0A20EE808A28EE080A60EE5E
:10582000080AB0EE680A08EE090A60EE80FAFAF794
:1058300049FF41EC1B0B1FEE900A01E056E0AAE085
:10584000FAF740FF41EC100B02F06EFB02F06CFB2C
:1058500053EC1B2B51EC100BFAF732FEFAF745FF15
:10586000D5ED0C1A9FED171AF0EE4F0A00EE100A54
:1058700041EEC10A08EE200AC8EE800A30EE890A1D
:1058800010EE100AFAF71EFF41EC100B02F04CFB71
:1058900002F04AFB53EC1C2B51EC100BFAF702FE02
:1058A000FAF723FF00EE100AB5F9420000EE900A65
:1058B000F8EEE00AF4EEC00AF1EE10FA18DD00206E
:1058C00031E00000339388430000000000000040F6
:1058D0000000204200FEFF46000080473333534063
:1058E0000000006066127140BD378635104629E71A
:1058F000B5F9440000EE900AF8EEE00AF4EEC00AB2
:10590000F1EE10FA01DD01200DE0B5F9460000EEE0
:10591000900AF8EEE00AF4EEC00AF1EE10FA01DDAA
:10592000022000E0032005EB800191ED0B1A05EB4E
:105930004001B1F9401000EE901A03A901EB80007C
:10594000F8EEE00A70EE600AB0EE4F0A01EE200AAF
:10595000D0ED000A60EE880A20EE200AC8EE800A28
:1059600030EE890A10EE100AFAF7ACFE41EC100B8B
:1059700002F0DAFA02F0D8FAB0EE4C1AF0EE6C1A35
:1059800053EC112B51EC100BFAF78CFDFAF7ADFE2E
:105990001C9941F82400641CB4F5407FFFF69AAED0
:1059A00008B000F003B805B000F006B8BDEC088BF5
:1059B000BDEC08CBFFF7F7BF30BCBDE8C08F0B468E
:1059C0004FF450724FF4105100F062B970B50C46AC
:1059D0000546FCF7E1F921462846FCF759F921462E
:1059E0002846FBF74DFE21462846FCF7B9F9B5F8E5
:1059F00070002146C0F3013084F824002846FBF7EC
:105A000047FE21462846FBF761FE21462846FBF764
:105A1000ABFC21462846FBF715FB21462846FCF740
:105A2000B1F821462846FBF7C1FE21462846FBF780
:105A3000CDFF21462846FBF743FC21462846BDE81A
:105A40007040FBF77DBD2DE9FC470D4681460024E3
:105A50004FF400466B4601223146484600F018F9E3
:105A600000282DD1BDF8000010F0080FF2D04FF43F
:105A700050774FF48068022C1ED2302231464846BF
:105A800000F02AF9411C1BD02B463A4641464846B5
:105A900000F0FEF8002813D16B460122314648463B
:105AA00000F0F6F800280BD1BDF8000004F1010465
:105AB00010F0080FE4B2DED1042C03D96FF0070018
:105AC00000F015B801AB012248F20D01484600F084
:105AD000DFF80100BDF80400A5F88006BDF800005D
:105AE00000F00100A5F88206EAD00846E8E70CBC01
:105AF000BDE8F08770B50C462DED068B054600F02D
:105B000065F8B5F84006B0EE409A00EE100A284954
:105B1000B8EE408A9FED270A18EE100A884201DD90
:105B200038EE408AB5F8000600EE900AF8EE608A7A
:105B300018EE900A884201DD78EEC08A9FED1E1BA8
:105B40009FED1F0B01F0B0FBB0EE40AA94ED040AEC
:105B5000F0EE60AA48EE008A88EE280A10EE100ADD
:105B6000FAF7B0FD53EC1A2BFAF7AAFCFAF7BDFDD1
:105B7000DFED150A94ED011A00EE100A79EE601AB5
:105B8000F7EE000AA08941EE210A80EE201A00EE0D
:105B9000100AD4ED020AB8EE400ABDEC068B31EED5
:105BA000400A80EE201AB3EE090A31EE000A70BDF9
:105BB00000FEFF4600008047000000000000324069
:105BC00000000000000000403333534010B50C4685
:105BD0002DED068BB0F85416284A00EE101AB8EED8
:105BE000408A18EE101A914203DD9FED250A38EE27
:105BF000408AB0F88006C0F38120FAF745FD9FED9A
:105C000021AB41EC110BB0EE4A0AF0EE6A0A01F04A
:105C10004BFBB0EE409AF0EE609A94F82400FAF74D
:105C200044FD41EC110BB0EE4A0AF0EE6A0A01F0B5
:105C30003BFBB0EE401AF0EE601A53EC192B51EC1E
:105C4000110BFAF7B2FCFAF750FD00EE100AB4F9A6
:105C5000020000EE900AB4F90000F8EEE00A50EEFF
:105C6000080A00EE100ABDEC068BB8EEC01A80EEF2
:105C7000810ADFED060A30EE200A10BD00FEFF4665
:105C80000000804700000000000000403333534014
:105C9000FEB516461D464FF6FF724FF4FA7302EA40
:105CA00046020095CDE9012340000A460146002442
:105CB00002230848FDF738FB38B1601EFEBD2819E5
:105CC0002A5D417842702955A41CB4EB460FF6DBDF
:105CD0000020FEBD386A00207FB505460E4640060E
:105CE000010E100A8DF80C0014468DF80D204FF4AB
:105CF000FA73022203A88DE80D00134632460B48C2
:105D0000FDF7C8FB18B14FF0FF3004B070BD084B71
:105D1000012231462846FFF7BBFF05480088A04214
:105D200002D06FF00100F0E70020EEE7386A0020B3
:105D3000040000202DE9F0432DED028B83B06E4F5F
:105D4000DFF8B881DFF8B8916EA001F04FFA76491C
:105D50003320FFF778FE010005D574A001F046FA64
:105D600000F086FAF0E780496F48FFF72FFF10EE4A
:105D7000104A7D496C48FFF7BDFEB0EE408ABCEE8C
:105D8000C80A10EE100AB87018EE100AFAF79AFC5A
:105D900005460E462046FAF795FC41EC100BCDE97E
:105DA000005653EC102B71A001F020FA74482044E7
:105DB000B0F5100F08D818EE100A404504D818EEB8
:105DC000100A704988421BDD18EE100AFAF77AFCB7
:105DD00005460E462046FAF775FC41EC100BCDE95E
:105DE000005653EC102B68A001F000FAF868401C34
:105DF000F8600528A8DB6BA001F0F8F901F042FA81
:105E00003D48B2EE000A801D78EE400AC07800EEF0
:105E1000100AB8EE401ADFED6E1A394A524981EE87
:105E2000210A4148FFF736FB4F4B012234496948AC
:105E3000FFF755FA67484C4B012231490A30FFF70A
:105E40004EFA0025644B2E462C46424648464FF4F7
:105E5000407C00BF00EB840191ED000A10EE101AA7
:105E6000914203D810EE101A99420CDD10EE100A80
:105E7000FAF728FC41EC100B214653EC102B57A0ED
:105E800001F0B4F90EE0E10726D000EE905AF8EEEA
:105E9000E00A30EE200ABDEEC00A10EE105A641C73
:105EA0006445D7DB1DB316B30124002002F0B8FD12
:105EB00002F0A1FE0146386158A001F097F95C4953
:105EC00038690968411A5BA001F090F903B02046D7
:105ED000BDEC028BBDE8F08300EE906AF8EEE00ABC
:105EE00030EE200ABDEEC00A10EE106AD7E757A0C8
:105EF00001F07CF928E7000010000020000020C21B
:105F00008C5700205B4D4C585D2053746172742097
:105F100072656164696E67206672616D6520646197
:105F200074610D0A000000008C6300205B4D4C582A
:105F30005D204661696C656420746F20676574201C
:105F40006672616D6520646174612C207374617484
:105F500075733D25642C207265747279696E672EA5
:105F60002E2E0D0A00000000A82B0020766464206D
:105F7000252E316620546120252E31660D0A000041
:105F80000000E0BF0000AA424661696C65642076AB
:105F9000646420252E316620546120252E31660D43
:105FA0000A0000005B4D4C585D204661696C6564D9
:105FB00020352074696D65732C2073797374656D59
:105FC00020726573657474696E670D0A00000000C5
:105FD0000000C8421856002000007F435B4D4C581B
:105FE0005D2054656D706572617475726520706FA7
:105FF000696E745B25645D20696E76616C69642CE2
:106000002076616C75653D252E31662C2072657495
:106010007279696E672E2E2E0D0A00004D4C585F66
:10602000656E645F7469636B20256C750D0A0000F2
:1060300008000020456C61707365642074696D65AB
:106040003A20256C75206D730D0A00005B4D4C588D
:106050005D204F6464206F72206576656E207375D5
:106060006D206973207A65726F2C20696E76616C81
:10607000696420646174612C207265747279696E40
:10608000672E2E2E0D0A0000F8B505464807860D2E
:1060900048F20D046B46012221462846FFF7F8FD21
:1060A000002808D1BDF80000214620F46072324378
:1060B0002846FFF711FEF8BD104810B50E490160E3
:1060C0000221416000214FF430228160C0E90312B7
:1060D0004FF4001242610176012242768276C27646
:1060E00001774277FCF7A3FA002803D0BDE81040FF
:1060F000FAF7A6BF10BD000000640040106A00203F
:10610000194808B5816C41F001018164816C01F08E
:1061100001010091816C41F002018164806C0022D8
:1061200000F00200009005211020FDF771FB102007
:10613000FDF761FB002205211120FDF769FB11200D
:10614000FDF759FB002205214420FDF761FB4420A7
:10615000FDF751FB002205214520FDF759FBBDE865
:1061600008404520FDF747BB0010024010B500F085
:10617000E1FB00F0C1FB114802F072FD104C0F4A28
:10618000012160621032084602F09EFD0B4AA062B7
:106190006C3A00210B4802F0E3FD084AA061483A3E
:1061A0000021094802F0DCFD044AE061243A0021A4
:1061B000064802F0D5FD206210BD0000C0A700080F
:1061C00010000020A96800088D6A00088B0E0008E6
:1061D0002DE9F04186B014216846FAF7B0F822485C
:1061E000C16C41F00401C164C16C01F0040105916E
:1061F000C16C41F00101C164C16C01F00101059164
:10620000C16C41F00201C164C06C184F00F0020083
:106210000590002248F211013846FCF7CAFF01221E
:1062200011033846FCF7C5FF4FF480764FF09048D5
:10623000002231464046FCF7BCFF49F211000090B5
:1062400001250024CDE90154694638460394FCF742
:10625000C5FE0096CDE90154694640460394FCF71B
:10626000BDFE06B0BDE8F081001002400004004809
:10627000134810B511490160124941600021012203
:10628000C0E90212016141618161C1610162FCF7F3
:10629000EFFF08B1FAF7D4FE00210948FCF794FF9C
:1062A00008B1FAF7CDFE00210548FCF7B8FF002839
:1062B00003D0BDE81040FAF7C3BE10BD0054004043
:1062C000386A00201A06100010B586B014216846FE
:1062D000FAF735F81D4800241B490594C0E900145D
:1062E0007F218160FF21C0E9031444618461C4619E
:1062F000FEF74CF908B1FAF7A3FE15208DF800005F
:106300008DF801408DF802400394012269460F4840
:106310000494FEF703FA08B1FAF792FE01208DF813
:1063200014008DF8150016208DF8160025208DF824
:106330001700012205A90548FEF7A0F9002801D0A1
:10634000FAF77EFE06B010BD002800401C6B00204E
:106350000D4810B50B4901604FF4E1314160002157
:1063600081600C22C160C0E904128161C1610162D7
:106370004162FEF7D3FC002803D0BDE81040FAF7D5
:106380005FBE10BD00440040406B0020FEE7FEE70A
:106390002DE9F04F2DED048B85B086A000F026FF8F
:1063A000DFF8408298ED008AF0EE488A9FED8E9AE1
:1063B0000024274620464FF4407100BF08EB8002BE
:1063C00092ED000AB4EEC80AF1EE10FA02DDB0EE6A
:1063D000408A06E0B4EE480AF1EE10FA02D1A0427B
:1063E00000DA0446B4EEE80AF1EE10FA02D2F0EE5A
:1063F000408A074630EE099A401C8842DEDB18EEE0
:10640000900AFAF75FF905460E4618EE100AFAF7F9
:1064100059F941EC100B02A9009481E8E00053EC1B
:10642000102B72A000F0E2FE9FED800ADFF80092D0
:106430000027C9EE000ABCEEC80A99F80050A9F17D
:10644000060310EE100AC1B2A94201D81F700FE076
:1064500010EE100AC0B2A84208D910EE100A99F83E
:106460000110C0B2884201D8012000E0022018705B
:106470001978DFF8BCB10BF1360B8BF8001010EE79
:10648000101ABCEEE80A8BF8011010EE101ABCEEE0
:10649000E00A8BF8021010EE101A8BF803109978AE
:1064A0008BF80410E01704EBD061481121F01F01B4
:1064B000611A002801DD421E00E00022172802DADE
:1064C00000F1010C01E04FF0170C002901DD4C1E1A
:1064D00000E00024A2461F2901DA4E1C00E01F261E
:1064E000534B00249B1F03F1440E5F649F641CE028
:1064F000534617E03B4F03EB421807EB8807012C8C
:1065000097ED000ABDEEC00A10EE107A04DA0BEB2C
:10651000040888F8077003E00EEB040808F8017C13
:106520005B1C641CB342E5DD521C6245E0DD8BF868
:1065300005108BF8060000215A46084673461C5C7D
:106540000CB9491CC9B2401C0828F8D3C91E03293C
:106550002ED9107820B1012807D002280ED027E0CC
:106560009BF80100A8420FD922E09BF801108D4250
:106570001ED299F80100814206D919E09BF801105A
:1065800099F80100814213D903F036F92848801F99
:10659000D0E90F12C0E90B12D0E91112C0E90D12B7
:1065A00003F04AF9012005B0BDEC048B00F042B8BD
:1065B0000020F8E75B50726F636573735D2053745E
:1065C0006172742070726F63657373696E67207493
:1065D000656D706572617475726520646174610DBA
:1065E0000A0000008C570020000000005B50726F12
:1065F000636573735D204D617854656D703D252E24
:106600003166206D6178496E6465783D25642C2083
:106610004D696E54656D703D252E3166206D696E35
:10662000496E6465783D25640D0A00000000404411
:106630001600002030BCBDE8C08F00002DE9F041FD
:10664000444C05468846E0680026810728680DD03E
:10665000E16801F00301814216D1A8B1E0686968E0
:10666000C0F30210401C88420ED120E0012804D063
:10667000022805D0032807D108E02168890701E036
:1066800021684905002907DB01265FE021688903AD
:1066900002D421684903F5E7E1686A686FF00F03E7
:1066A00021F0730103EB021211430143E160206802
:1066B00020F080602060FCF781FD074605E000BF08
:1066C000FCF77CFDC01B022837D820680001F7D4F6
:1066D000B8F1000F18D0B8F1010F1DD0287D4FF090
:1066E0007E41400801EB4060A96840EA0120216931
:1066F000194A114008432061206840F08060206002
:10670000FCF75CFD07461AE0A868297B000240EA16
:10671000C1602169114AECE7288A1149400801EB60
:106720004050A96840EA012021690E4AE1E700BF14
:10673000FCF744FDC01B022801D9032606E02068AF
:106740000001F5D52069A969084320613046BDE8FC
:10675000F081000000100240FF80FFF9FF80FF077A
:106760000000E0FFFF809FFFF8B51C4D06460024A7
:10677000A86DC00002D5FDF7CDF80DE0A86D40F082
:106780008050A865A86D00F080500090FDF7C2F819
:10679000A96D21F08051A965B0F5007F04D0802E4D
:1067A00007D94FF003040AE0802E08D9A02E01D8A3
:1067B00004E001D1022402E0702E00D10124084837
:1067C000016821F0070121430160006800F0070023
:1067D000A04201D00120F8BD0020F8BD0010024009
:1067E000002002400022014602E00A39C9B2521CD0
:1067F0000A29FAD2100741EA106070472DE9F041EA
:10680000044600680025C168490617D4691EC160A6
:10681000FCF7D4FC06464FF47A78032708E000BF63
:10682000FCF7CCFC801B404502D9032584F821707D
:106830002068C068400601D4032DF1D12846BDE888
:10684000F08100002DE9F04106461348002501685B
:1068500021F080010160041F20684FF003078006CB
:1068600007D43046FDF7C0FF90B186F821700325AC
:106870000EE0206820F0200020603046FDF7B4FFD5
:1068800010B186F821700325206840F020002060B8
:106890002846BDE8F08100000C2800400148FDF7C3
:1068A0005BBE00001C6B00200EB503F0A3FD019041
:1068B00000208DF808000F4CCDF80000FFF73AFAE1
:1068C000A0B1FFF765FD012810D1694601A8FAF7CC
:1068D000C1F8206880694007F0D4694602A8FAF739
:1068E0009FFA0098401C0090FAF78CFB0A2002F0F7
:1068F00075F9E3E7106A0020054801780548FF298B
:10690000818001D12D21818089B203A000F06EBC6D
:1069100000880108100000204C6F616465642064E9
:106920006174613A204E4F44455F49443D25750AE4
:106930000000000008B50F490F480A78FF2A00D16F
:106940003C2202704A78FF2A00D1642242708A7881
:10695000FF2A00D11E228270C978FF2900D15F2151
:10696000C170C9B20091837842780178034800F081
:106970003DFC08BD00FC010816000020B8A8000876
:106980001CB5002100918DF8000001AB042269467E
:106990000648FBF75BFB18B105A000F027FC1CBD07
:1069A0009DF800100BA000F021FC1CBD0088010820
:1069B0004661696C656420746F2073617665204E52
:1069C0004F44455F494420746F20666C6173680AC8
:1069D000000000004E4F44455F49442073617665D6
:1069E0006420746F20666C6173683A2025750A0014
:1069F0000EB58DF804008DF805108DF806208DF881
:106A0000073002AB042201A90A48FBF71FFB18B1AB
:106A100009A000F0EBFB0EBD9DF8070000909DF86B
:106A200006309DF805209DF804100CA000F0DEFB58
:106A30000EBD000000FC01084661696C65642074AD
:106A40006F207361766520506172616D6574657247
:106A500020746F20666C6173680A00005061726177
:106A60006D6574657220736176656420746F20664D
:106A70006C6173683A205B25755D205B25755D2030
:106A80005B25755D20205B25755D0A00642002F0A2
:106A9000A5F8FBE710B54FF0E020006903F09CFC7F
:106AA000012803D0BDE8104003F050B910BD00002C
:106AB00000B597B044216846F9F741FC142111A8AC
:106AC000F9F73DFC4FF40070FCF7D4FE08B172B644
:106AD000FEE7FCF727FF194850F8901F21F0180136
:106AE00001600E20012100900802CDE90210102063
:106AF000CDE9040102200A90CDE90B0108210D9196
:106B00000721CDE90E1010906846FDF7A9F908B1EC
:106B100072B6FEE70F201190032012909020139080
:106B2000002014900146159011A8FDF761F8002887
:106B300001D072B6FEE717B000BD000000100240A1
:106B40000248016841F470010160704788ED00E07F
:106B50000148FDF7C6BE0000546C002070B5026805
:106B6000164B4FF08046984201D0B04203D122F03C
:106B700070044A682243124C124D984205D0B0422C
:106B800003D0A04201D0A84203D122F44076CA68C3
:106B900032434E6922F08002324302608A68C26248
:106BA0000A688262984203D0A04201D0A84201D173
:106BB000096901630121416170BD0000002C0140A1
:106BC000004001400044014090F82410C90706D05D
:106BD00001684A68836A22F400321A434A6090F8D6
:106BE0002410890706D501684A68C36A22F48032F6
:106BF0001A434A6090F82410490706D501684A688C
:106C0000036B22F480221A434A6090F8241009078B
:106C100006D501684A68436B22F400421A434A6071
:106C200090F82410C90606D501688A68836B22F49F
:106C300080521A438A6090F82410890606D50168AC
:106C40008A68C36B22F400521A438A6090F82410B9
:106C5000490611D501684A68036C22F480121A4370
:106C60004A60016CB1F5801F06D101684A68436C27
:106C700022F4C0021A434A6090F82410090606D58F
:106C800001684A68806C22F4002202434A6070471F
:106C9000F8B500260446C0F88060FCF78FFA054678
:106CA000206800686FF07E47000708D52B46002259
:106CB0004FF400112046009700F01AFA60B92068DE
:106CC000006840070AD52B4600224FF48001204679
:106CD000009700F00DFA08B10320F8BD2020A0674E
:106CE000E067266684F874600020F8BD10B5806AFD
:106CF0000021A0F85A10A0F85210FDF7C4FE10BDF4
:106D000070B5846AA06FE56F216889684FF000064E
:106D1000090606D5212804D1A4F85260204600F0C7
:106D200088F820688068400606D5222D04D1A4F892
:106D30005A60204600F058F8D4F8800040F0100067
:106D4000C4F880002046FDF79EFE70BD10B50146D8
:106D5000806A0968096889062DD40021A0F85A10B4
:106D6000016851E8002F22F4807241E80023002BD3
:106D7000F6D10168083151E8002F22F0010241E804
:106D80000023002BF5D10168083151E8002F22F0D3
:106D9000400241E80023002BF5D12021C167016E9C
:106DA000012908D1026852E8001F21F0100142E8D1
:106DB0000013002BF6D1016E012902D0FEF786F8F0
:106DC00010BDB0F85810FDF75CFE10BD10B5806A1C
:106DD000016E012902D0FEF77AF810BDB0F8581004
:106DE0004908FDF74EFE10BD016851E8002F22F45E
:106DF000907241E80023002BF6D10168083151E878
:106E0000002F22F0010241E80023002BF5D1016E92
:106E1000012908D1026852E8001F21F0100142E860
:106E20000013002BF6D12021C167002101664166C5
:106E30007047026852E8001F21F0C00142E80013C9
:106E4000002BF6D120218167704700002DE9F04129
:106E50000446016880682269E3691043626900257D
:106E60001A431043714F0A68714B1A4002430A607B
:106E700020684168E26821F4405111434160216873
:106E8000A069B94201D0226A10438A6822F43062B4
:106E900002438A606749236867488B420DD1D0F866
:106EA000880010F0030006D0012847D0022843D004
:106EB000032830D144E001212EE060498B420BD100
:106EC000D0F8880010F00C0034D0042836D0082800
:106ED00032D00C281FD133E059498B420BD1D0F866
:106EE000880010F0300025D0102827D0202823D08B
:106EF000302810D124E0BB420DD1D0F8880010F426
:106F0000406017D0B0F5806F18D0B0F5006F13D087
:106F1000B0F5406F14D010214A4A00264FF40040CB
:106F2000BB422FD171B102290FD004290FD00829FB
:106F300073D10FE00021EFE70221EDE70421EBE739
:106F40000821E9E7FCF716FF03E0104602E0FCF732
:106F500035FFE8B3626802EB420181425DD8B0EBD5
:106F6000023F5AD8010E030250081818714100233D
:106F7000F9F798F9344AA0F5407191424DD821684B
:106F8000C8604BE0E3694FF6EF77834228D10929C7
:106F900043D2DFE801F005080B420D4242421000E7
:106FA000FCF7E8FE06E0FCF7F7FE03E0104602E01F
:106FB000FCF704FF60B14100606801EB5001B1FBD8
:106FC000F0F0A0F11001B94227D84FF6F07100E0BF
:106FD00024E00140C0F3420001432068C1601DE08D
:106FE00009291AD2DFE801F005080B190D19191942
:106FF0001000FCF7BFFE06E0FCF7CEFE03E01046F3
:1070000002E0FCF7DBFE48B1616800EB5100B0FB29
:10701000F1F0A0F11001B94205D9012566662846B4
:10702000A666BDE8F08180B2A9E7000000800040BC
:10703000F369FFEF003801400010024000440040B7
:10704000004800400024F400FFFC0F0070B54165CB
:10705000A0F8582000250446C0F880502220E067A0
:10706000206FD8B11F49C162216F1F4813460863C2
:10707000216F1E484863206F8563666D2168324624
:107080002431206FFBF7DAFD40B11020C4F88000F6
:1070900004F8745F2020A060012070BD84F8745053
:1070A000206940B1216851E8000F40F4807041E848
:1070B0000002002AF6D12068083050E8001F41F095
:1070C000010140E80012002AF5D12068083050E89C
:1070D000001F41F0400140E80012002AF5D10020D5
:1070E00070BD00004D6D0008CD6D0008016D0008F9
:1070F0002DE9F0479A4617460E4604464FF0000920
:107100004FF02008089D4AE0681C48D0FCF756F86C
:10711000A0EB0A00A8422AD84DB3206801684907AD
:107120003DD5C069C043000539D421684FF40060E3
:107130000862206850E8001F21F4D07140E8001276
:10714000002AF6D12068083050E8001F21F0010124
:1071500040E80012002AF5D1C4F87880C4F87C8099
:10716000C4F8808084F874900320BDE8F08721681B
:1071700051E8000F20F4D07041E80002002AF6D157
:107180002068083050E8001F21F0010140E800129B
:10719000002AF5D1C4F87880C4F87C80E2E7206842
:1071A000C06936EA000004D00020B842ACD000200C
:1071B000DBE70120F9E70000094810B50068C16964
:1071C000C943C90606D410210162092205490448B1
:1071D000FDF752FEBDE810400148FDF755BC000028
:1071E000406B00201C250020FEE700000FB4054B7B
:1071F00010B503A9044A029801F072F810BC5DF8BA
:1072000014FB0000498A00080C0100200FB4084B51
:1072100010B504A902AA039801F062F8044602A975
:10722000002001F0F7FB204610BC5DF814FB0000C5
:10723000158A000803B401984100009850EAC12063
:1072400018BF04204A0D18BF40F0010040F2FF7241
:10725000B2EB515F08BF40F00200012808BF0520D3
:1072600002B070470907090E002804DB00F1E02096
:1072700080F80014704700F00F0000F1E02080F863
:10728000141D7047BFF34F8F05480168054A01F48C
:10729000E06111430160BFF34F8F00BFFDE70000C5
:1072A0000CED00E00400FA052DE9F04D2DED040B86
:1072B0002DED0E8B96B0DDE92550279CDDF890A0D2
:1072C00025F0004624F00048BAF1000F14BF012158
:1072D000002101EB4502FC4953184A1093422AD37E
:1072E000002814BF0123002303EB44030B44F74998
:1072F0008B4220D358EA00019FEDF59B76D0DFF852
:10730000D8B35D4503D1BAF1000F05D188E0BAF1D9
:10731000000F08BF002100D0012101EB450111F54C
:10732000001F08D8002814BF0121002101EB4401EF
:1073300011F5001F0BD99DED261B9DED240B16B0FA
:1073400000F0DABD04B0BDE8F04D00F0C1BE00278A
:10735000002DBCBFE149884521DAE1498845A8BF35
:1073600002271CDAC3451ADCDE4901EB2851142937
:1073700008DDC1F1340220FA02F101FA02F2824280
:107380000DD108E058B9C1F1140228FA02F101FA4E
:1073900002F2424503D101F00101C1F1020756EAB0
:1073A0000A0124D1002C22DA002D18BF022F01D0AF
:1073B000012F0AD0022000F0D7FE16B000F0A2BDC7
:1073C00004B0BDE8F04D00F06BBE022000F0CCFE32
:1073D00000F066FE51EC100B81F0004141EC100B07
:1073E00016B000F095BD04B0BDE8F08D18E09FED3B
:1073F000BEAB9FEDBF8B002871D1B848804522D12C
:1074000005F1804010F5801008BFBAF1000F07D0D9
:10741000B3450ADC002CA8BF9DED260BE0DA0DE099
:10742000B0EE490AF0EE690ADAE7002C06DA9DEDC3
:10743000260B51EC100B81F000416FE0AE48784410
:1074400090ED000BCCE7D8454DD1002C48DA2EB199
:1074500086423AD1BAF1000F42D126E0BAF1000FCC
:1074600013D0022000F080FE00F04EFE8DED020BE6
:107470009DED240B8DED000B10EE900A039961F346
:107480001E0003909DED020BAAE78DED02AB9DED72
:10749000240B1AEE901A10EE900A8DED000B61F39A
:1074A0001E0003909DED020B9AE78DED028B9DED82
:1074B000240B18EE901A10EE900A8DED000B61F37C
:1074C0001E0003909DED020B8AE709DA9DED240B67
:1074D00051EC190B53EC102BF9F767F81EE020E084
:1074E0009DED240B7CE786421BDAB4F1804F0DD072
:1074F000A4F10050B0F1FF5013D1002D11DB9DED30
:10750000240B51EC100B02F0CDF807E09DED240B9D
:1075100053EC102B51EC100B00F0C2BC41EC100BE3
:107520005EE79DED240B51EC100B01F081FABAF1EE
:10753000000FCDE90E0142D19FED710B46B3A6F1CC
:10754000E040B0F17F600CD05E4538D1002D00DA0C
:10755000A7B3022F0CBF01204FF0FF30F9F794F8CA
:10756000DCE7002D01DD002C0DDA002D01DD002C03
:107570001FDB002D16DA002C14DB012F08BF9FED56
:10758000620B3FF42DAFB0EE4A0AF0EE6A0A27E72D
:10759000022F18BF002D0CD0012F0AD1002DFFF6AD
:1075A0001FAF06E0002DB8BF002C08DA012F3FF412
:1075B00017AFB0EE480AF0EE680A11E71BE00120B1
:1075C00000EBE57050EA070115D0791EB0EE498A4C
:1075D000F0EE698A084308BF9FED4D8B4E480025A9
:1075E000804570DD4D494E48884514DDB0420DDBC5
:1075F000002C19DB2FE0012000F0B6FD16B000F0E2
:107600008DBC04B0BDE8F04D00F06EBDB34502DCAA
:10761000002C09DC1FE0864202DA002C1BDA03E0B2
:107620005E452BDD002C16DD022000F09DFD00F0F4
:107630006BFD8DED020B53EC1A2B51EC180BF8F788
:107640003FFFCDE900010399019861F31E0003900B
:107650009DED020BC4E6022000F086FD00F064FD03
:1076600010EE901A18EE900A8DED020B8DED008B46
:1076700061F31E0003909DED020BB1E69DED0E0B34
:1076800053EC192B51EC100BF8F70CFF9FED260B68
:10769000CDE9080153EC102B9DED080B51EC100BBC
:1076A000F8F70EFF9FED221B53EC112BF8F7FDFEB0
:1076B0009DED081B53EC112BF8F702FF9FED1E1BED
:1076C00053EC112B3CE08CE0FFFF1F00FFFF0F008D
:1076D000000000000000F03F0000F03F0000F07FDD
:1076E0000000404301FCFFFF000000000000F07FAD
:1076F00000000000000000006E34000000000000E8
:107700000000000000000080000000000000F0FF0A
:10771000000000000000F0BF0000E0410000F04366
:10772000FFFFEF3F00000000000000000000D03F1E
:10773000555555555555D53F000000000000E03F18
:10774000F8F7B3FE9DED080B41EC1A0B53EC102B30
:1077500051EC100BF8F7B4FE53EC1A2BF8F7B0FE0F
:1077600041EC1A0B9FEDFE0B53EC102B9DED080B1B
:1077700051EC100BF8F7A4FE41EC1B0B9FEDFA0B3C
:1077800051EC1A0B53EC102BF8F79AFE41EC1A0B44
:107790009FEDF70B53EC102B9DED080B51EC100BEC
:1077A000F8F78EFE53EC1A2BF8F77CFE41EC1A0B1F
:1077B00051EC1B0B53EC1A2BF8F7D3FD0690CDE9D7
:1077C00006519DED060B53EC1B2B51EC100BF8F7FB
:1077D00069FE53EC1A2BF8F768FE41EC100B00F031
:1077E000A1B90020B6F5801F0EDA9FEDE30B53EC34
:1077F000102B9DED0E0B51EC100BF8F761FECDE94F
:107800000E016FF034000E4600EB2650A0F2FF3759
:10781000C6F31300DA4940F07F6646F040568842CE
:10782000D8BF002408DDD7498142C8BF012403DC4A
:107830000024A6F580167F1CD348784400EBC400D2
:107840000F9690ED00CB9DED0E0B53EC1C2B51ECE5
:10785000100BF8F727FE9DED0E0B41EC1B0B53ECC4
:107860001C2B51EC100BF8F77CFD41EC100B51EC8C
:10787000190B53EC102BF8F798FE41EC1D0B51EC53
:107880001B0B53EC1D2BF8F71BFE41EC1A0BBF48EA
:107890008DED10AB7844109590ED000B4FF000503B
:1078A00040EA660000EB84408DED080B00F50020F7
:1078B00009909DED080B53EC1C2B51EC100BF8F7C5
:1078C000F1FD9DED0E1B53EC112BF8F7EEFD41EC95
:1078D000100B53EC102B9DED100B51EC100BF8F727
:1078E000EFFD9DED080B41EC1C0B53EC102B9DEDB7
:1078F000100B51EC100BF8F7E3FD53EC1B2BF8F7D2
:10790000D4FD53EC1C2BF8F7CDFD53EC1D2BF8F7F1
:10791000D7FD41EC1C0B53EC1A2B51EC1A0BF8F76A
:10792000CFFD41EC1B0B9A480621B0EE4B0AF0EE5E
:107930006B0A784400F035FBB0EE401AF0EE601AA6
:10794000B0EE41DAF0EE61DA53EC1B2B51EC1B0B7D
:10795000F8F7B6FD53EC1D2BF8F7B2FD9DED100BBB
:1079600041EC1B0B53EC1A2B51EC100BF8F7F9FC04
:1079700053EC1C2BF8F7A4FD53EC1B2BF8F7F1FC90
:107980009DED100B41EC1B0B53EC102B51EC100B2D
:10799000F8F796FD41EC1D0B9FED7FEB53EC1E2B92
:1079A000F8F7DFFC53EC1B2BF8F7DBFC0890CDE974
:1079B00008519DED080B53EC1E2B51EC100BF8F702
:1079C00071FD53EC1D2BF8F76DFD53EC1B2BF8F7F5
:1079D0006CFD9DED080B41EC1D0B53EC102B9DED48
:1079E000100B51EC100BF8F76BFD41EC1B0B53EC3B
:1079F0001A2B51EC1D0BF8F763FD9DED080B41ECC4
:107A00001A0B53EC102B51EC1C0BF8F759FD53ECEF
:107A10001A2BF8F7A6FC41EC1A0B51EC1B0B53EC9C
:107A20001A2BF8F79EFC0C90CDE90C519DED0C0B38
:107A300053EC1B2B51EC100BF8F734FD53EC1A2BC5
:107A4000F8F733FD41EC1B0B9FED550B53EC102B5E
:107A50009DED0C0B51EC100BF8F732FD41EC1A0BBD
:107A60009FED510B51EC1B0B53EC102BF8F728FD3D
:107A700041EC1B0B9FED4E0B53EC102B9DED0C0BB3
:107A800051EC100BF8F71CFD53EC1B2BF8F769FCBD
:107A900041EC100B4848784400EBC40090ED001B0B
:107AA00051EC100B53EC112BF8F75BFC41EC1B0B6A
:107AB0003846F8F7E9FDCDE9080153EC1B2B51ECF2
:107AC0001A0BF8F74EFC41EC100B3C48784400EBE5
:107AD000C40090ED00CB51EC100B53EC1C2BF8F7CD
:107AE00040FC9DED081B53EC112BF8F73AFC069077
:107AF000CDE906519DED080B53EC102B9DED060BC7
:107B000051EC100BF8F7CEFC53EC1C2BF8F7CAFC29
:107B100053EC1A2BF8F7C6FC53EC1B2BF8F7C5FCFB
:107B200041EC100B9DED261B53EC102B8DED001B33
:107B300000959DED260B51EC100BF8F7C1FC9DED67
:107B4000000B41EC1A0B53EC102B9DED260B51EC66
:107B5000100BF8F7A7FC9DED061B53EC112B2FE043
:107B6000000000604715F73FFE822B654715F73F81
:107B700044DF5DF80BAE543E0000000000004043BF
:107B80008E9803007AB60B00EA2F00001830000030
:107B9000222F00000000000000000000000008404C
:107BA000000000E009C7EE3FFD033ADC09C7EE3FE5
:107BB000F5015B14E02F3EBEAE2D0000682D0000E5
:107BC000F8F77EFC53EC1A2BF8F7CBFB9DED060B78
:107BD00041EC1A0B53EC102B9DED000B51EC100BEC
:107BE000F8F76EFCCDE90C019DED0C0B51EC1A0B76
:107BF00053EC102BF8F7B5FBCDE902010C46AA496E
:107C00008C422FDB611A084318D19DED0C0B53EC0D
:107C1000102B9DED020B51EC100BF8F743FC41ECDF
:107C20001B0B9FEDA30B51EC1A0B53EC102BF8F729
:107C300098FB53EC1B2BF8F7CFFE2DD2022000F05F
:107C400093FA00F061FA10EE901A18EE900A8DED9A
:107C5000020B8DED008B61F31E0003909DED020B76
:107C6000FFF7BEBB944A24F00041914214D39349DC
:107C7000214408437FF4EFAC9DED0C0B53EC102B2B
:107C80009DED020B51EC100BF8F70CFC53EC1A2B8A
:107C9000F8F7A2FE7FF6DFAC24F000408849894A5D
:107CA000002601EB205182422BDA481C4FF4801150
:107CB00021FA00F02044844AC0F30A517A44A1F228
:107CC000FF3192ED000B814A8DED080BCA4020EA8E
:107CD0000202C0F3130040F48010C1F1140120FA35
:107CE00001F60992002CB8BF76429DED080B53ECCB
:107CF000102B9DED0C0B51EC100BF8F7D3FBCDE9DD
:107D00000C019DED0C0B51EC1A0B53EC102BF8F7FA
:107D100028FB9FED6F0B0890CDE9085153EC102B19
:107D20009DED080B51EC100BF8F7CAFB41EC1B0B57
:107D30009FED690B53EC102B9DED080B51EC100BD4
:107D4000F8F7BEFB9DED0C0B41EC1C0B53EC102B1C
:107D50009DED080B51EC100BF8F7A4FB53EC1A2B1C
:107D6000F8F7A3FB9FED5E1B53EC112BF8F7A8FB74
:107D700053EC1C2BF8F7F5FA41EC1A0B51EC1B0BEA
:107D800053EC1A2BF8F7EDFACDE902019DED020B49
:107D900053EC1B2B51EC100BF8F784FB53EC1A2B14
:107DA000F8F783FB9DED020B41EC1A0B53EC102B03
:107DB00051EC100BF8F784FBCDE908014A489DED22
:107DC000080B0521784400F0ECF89DED081B51EC00
:107DD000100B53EC112BF8F773FB9DED021B53ECCA
:107DE000112BF8F762FBCDE906019DED020B53EC78
:107DF0001A2B51EC100BF8F763FB53EC1A2BF8F726
:107E0000B0FA9FED3B0B41EC1A0B53EC102B9DEDA0
:107E1000060B51EC100BF8F745FB9DED060B41EC02
:107E20001B0B53EC102B9DED020B51EC100BF8F7D4
:107E300047FB53EC1B2BF8F7B8FB53EC1A2BF8F766
:107E400031FB9DED021B53EC112BF8F72BFB53EC90
:107E5000192BF8F72AFBCDE9020101EB06500115B9
:107E60000029C8BF039015DC9DED020B324651EC92
:107E7000100BF8F731FDFFF7DDF9042808BF00F01B
:107E800053F932469DED020B51EC100BF8F724FD2F
:107E9000CDE902019DED020B51EC180B53EC102BB8
:107EA000F8F70EFBFFF73ABB00009040000000001F
:107EB000FE822B654715973C00CC904000346F3F05
:107EC00001FCFFFF0000E03FF02B0000FFFF0F0070
:107ED00000000000432EE63F396CA80C615C20BE18
:107EE000EF39FAFE422EE63FC02A000000000000F3
:107EF0000000000000000040BDEC088BBDEC06CB8C
:107F0000FFF720BABDEC088BBDEC06CBFFF758BAE3
:107F1000BDEC088BBDEC06CBFFF765BABDEC088B5A
:107F2000BDEC06CBFFF76DBB00B52DED048BB0EEBD
:107F3000409AF0EE609A83B051EC190BF8F7E3FC2D
:107F400041EC180B18EE100A18EE901A8DED008B0C
:107F5000002818BF0120084320F00040C0F17F60D6
:107F600000F1E040C00F14D019EE101A19EE900A7B
:107F70008DED009B002918BF0121084320F000402F
:107F8000C0F17F6000F1E040C00F04BF012000F0AD
:107F9000EBF8B0EE480A03B0F0EE680ABDEC048BD3
:107FA00000BD70B504462DED028B4D1E00EBC500E3
:107FB000B0EE408AF0EE608A90ED000B35F00600DE
:107FC00017D053EC182B51EC100BF8F779FA41EC61
:107FD000100B6D1E04EBC50090ED001B51EC100B57
:107FE00053EC112BF8F7BDF941EC100B35F00600FE
:107FF000E7D1022D36D0042D1CD0062D1CBFBDECC0
:10800000028B70BD53EC182B51EC100BF8F758FA9B
:1080100094ED0A1B53EC112BF8F7A3F953EC182B32
:10802000F8F74EFA94ED081B53EC112BF8F799F979
:1080300041EC100B53EC182B51EC100BF8F740FAF5
:1080400094ED061B53EC112BF8F78BF953EC182B1E
:10805000F8F736FA94ED040B53EC102BF8F781F98E
:1080600041EC100B53EC182B51EC100BF8F728FADD
:1080700094ED021B53EC112BF8F773F953EC182B0A
:10808000F8F71EFA94ED001B53EC112BF8F769F981
:10809000BDEC028B41EC100B70BD00000000000035
:1080A0009FED070B10B553EC102B9FED070B51EC18
:1080B000100BF8F77AFA41EC100B10BD000000002D
:1080C0000000000000000000000000000000F03F81
:1080D00010B553EC112B51EC100BF8F742F941ECB1
:1080E000100B10BD000000009FED050B10B553EC08
:1080F000102B51EC100BF8F758FA41EC100B10BD97
:1081000000000000000000009FED050B10B553ECCF
:10811000102B51EC100BF8F7D3F941EC100B10BDFC
:1081200000000000000000709FED050B10B553EC3F
:10813000102B51EC100BF8F7C3F941EC100B10BDEC
:10814000000000000000001002E008C8121F08C173
:10815000002AFAD170477047002001E001C1121FC8
:10816000002AFBD1704700000149086070470000F9
:10817000180100202DE9FF5FDDE90220010DDDF887
:1081800038B0024318D044F61050A1F2FF314143F9
:108190000D140F98012820D0A5EB0B00401C5FEABE
:1081A000000A4FF00004474EDFF81C91A0465046ED
:1081B00016D5CAF1000728E00F98012443A2012830
:1081C00008D0002100980F9BC0E90021C0E90243BC
:1081D00000F082B86FEA0B01F4E7CBF10000DEE7B4
:1081E000074612E0F80707D0224633464046494684
:1081F000F8F766F980468946224633461046194606
:10820000F8F75EF904460E467F10002FEAD1DDE94B
:108210000201BAF1000F42464B4602DAF8F750F974
:1082200001E0F8F7C2F904460E460022284BF8F7A1
:10823000D3FB03D84FF0FF30014607E00022254B67
:1082400020463146F8F78DF8F8F7AEFB102409E028
:10825000002C0ADB0A220023F8F724F8019B3032B5
:108260001A55641E50EA0102F2D1641C019AC4F14D
:10827000110314440F9A012A03D0012208430DD19F
:108280000AE0084304D000204FF0110B0F9080E764
:10829000A3EB0B056D1E0DE05B4504DD4FF0000206
:1082A00005F1010504E003DA4FF00002A5F1010534
:1082B000002AECD000980F99C0E90231C0E90045CE
:1082C00086E70000000024400000F03F300000007E
:1082D0000000F0430000E03F3FBCBDE8C09F00004D
:1082E0002DE9FF4F95B09B468946064600250FE2D3
:1082F000252877D100242746F84A0121059400E07B
:10830000044316F8013F203B01FA03F01042F7D175
:1083100030782A2811D06FF02F033078A0F1300286
:10832000092A16D8059A44F0020402EB820203EBF4
:1083300042021044761C0590EFE759F8042B059291
:10834000002A03DA504244F40054059044F0020439
:10835000761C30782E2816D116F8010F44F004044C
:108360002A280DD06FF02F023078A0F13003092BAE
:1083700009D807EB870302EB4303C718761CF3E722
:1083800059F8047B761C30786C280FD006DC4C281A
:1083900017D068280DD06A2814D104E0742810D0B2
:1083A0007A280FD10DE044F400140AE044F480145C
:1083B00001E044F440147278824202D104F5801442
:1083C000761C761C307866280BD013DC582877D0C2
:1083D00009DC002875D04528F6D04628F4D0472877
:1083E0001AD19DE118E0632835D0642879D065283A
:1083F00012D195E1702873D008DC6728F1D0692884
:108400006FD06E280DD06F2806D1B5E073282CD020
:10841000752875D0782874D05A46179990476D1CE6
:1084200075E1C4F30250022809D003280DD0D9F811
:10843000001004280DD00D6009F1040967E1D9F896
:108440000010EA17C1E90052F6E7D9F800100D80D4
:10845000F2E70D70F0E719F8041B8DF8001000200A
:108460008DF80100EA46012003E059F804AB4FF013
:10847000FF3061074FF0000102D40DE008F1010167
:108480008846B9420FDA8045F8DB1AF8081000294F
:10849000F4D108E008F1010188468142FADB1AF8BC
:1084A00008100029F6D105985B46A0EB0807214685
:1084B0003846179A00F097FA284400EB080507E0C1
:1084C0004DE029E10DE01AF8010B5A461799904743
:1084D000B8F10108F7D25B4621463846179A13E1F6
:1084E00042E00A220092C4F302524FF0000A022A2C
:1084F00008D059F804CB032A4FEAEC710AD00DE0FA
:1085000029E02AE009F1070121F00702F2E802C19F
:10851000914609E00FFA8CFC4FEAEC71042A03D172
:108520004FFA8CFC4FEAEC71002907DA0A46002169
:10853000DCF1000C61EB02012D2202E0220504D5E2
:108540002B228DF80420012203E0E20701D0202233
:10855000F7E7904659E00A2102E010220DE01021D1
:108560004FF0000A00910BE010224FF0000A44F097
:1085700004040827009203E008224FF0000A00924A
:10858000C4F30252022A05D059F804CB0021032A71
:1085900008D009E009F1070121F00702F2E802C161
:1085A000914605E01FFA8CFC042A01D10CF0FF0C67
:1085B0004FF00008220728D5702806D0009B83F0D2
:1085C000100353EA0A0305D00EE040228DF8042080
:1085D000012208E05CEA010206D030228DF8042076
:1085E0008DF8050002229046009B83F0080353EAB1
:1085F0000A030AD15CEA010201D1620705D53022E3
:108600008DF804204FF001087F1E582804D034A0B4
:1086100003900EA802900DE036A0F9E7534660469D
:10862000009AF7F73FFE84460398825C0298401E4A
:10863000029002705CEA0100F0D1029806A9081AC3
:1086400000F1200A600702D524F4803400E00127FD
:10865000574502DDA7EB0A0000E0002000EB0A010D
:10866000009005984144401A0590E00306D45B460B
:108670002146179A059800F0B6F90544002706E050
:1086800001A85A46C05D179990476D1C7F1C47454D
:10869000F6DBE0030CD55B462146179A059800F0FF
:1086A000A2F9054404E030205A46179990476D1C02
:1086B0000099481E00900029F5DC08E00298029914
:1086C0005A460078491C0291179990476D1CBAF1DF
:1086D0000001AAF1010AF1DC65E1000009280100AE
:1086E0003031323334353637383961626364656628
:1086F00000000000303132333435363738394142EA
:10870000434445460000000000F05BF90544761C38
:10871000307800287FF4ECAD19B0284600F04EB94F
:10872000620700D4062709F1070222F0070CFCE8D3
:108730000223E14603F000485FEA080C02D00FF282
:10874000702C0DE05FEA045C02D50FF2682C07E0A4
:108750005FEAC47C02D00FF2602C01E0AFF2700C33
:108760004FF0FF3823F00043CDF850C065280CD0FF
:1087700006DC452809D046281DD047283DD13DE0DC
:10878000662818D067287ED138E00021112F01DB40
:10879000112000E0781CCDE9000106A90EA8FFF722
:1087A000E9FCDDE90F010E9A03910021009207F127
:1087B000010A04914DE04FF000400097CDE901100F
:1087C00006A90EA8FFF7D6FCDDE90F0203920E9B67
:1087D00011990022DDF80CA00093049211B9791CC4
:1087E00000EB010AB7EB0A0004D4C0F1FF3007F137
:1087F000010A0490AAEB0700019044E0012F00DA7F
:1088000001270021112F01DD112000E03846CDE9BC
:10881000000106A90EA8FFF7ADFCDDE90F010E9AD5
:108820000391002104910092BA4621070CD40399C8
:10883000514500DA8A46BAF1010F05DD009AAAF126
:108840000101515C302908D0B84202DA10F1040F5E
:1088500006DA0121CDE9011015E0AAF10101E9E7ED
:10886000002805DC049901440491AAEB000102E010
:10887000411C514500DD8A460499401A401C019074
:108880004FF000400290200704D40198504501DBCE
:10889000CDF8048000208DF84F0002980DF14F07AD
:1088A000B0F1004F25D02B200E9002984FF0020817
:1088B00000280CDA404202902D200E9007E00A2199
:1088C0000298F7F72EFF3031029007F8011DB8F13A
:1088D0000001A8F10108F2DC02980028EFD1791E0E
:1088E0000E980870307800F0200040F0450007F83E
:1088F000020D12A8C01B00F107081498007800B1FF
:10890000012000EB0A01019801EBE0710598414458
:10891000401A401E0590E00306D45B462146179A94
:10892000059800F060F805441498007818B15A468C
:10893000179990476D1CE00324D55B462146179A92
:10894000059800F050F805441CE00498002807DB67
:10895000DDE90301884203DD0098405C179901E0DE
:10896000179930205A469047049805F10105401C9C
:1089700004900198401E019004D12E205A46179968
:1089800090476D1CBAF10001AAF1010ADDDC05E097
:1089900017F8010B5A46179990476D1CB8F1000162
:1089A000A8F10108F4DC5B462146179A0598ABE66E
:1089B0002D0000002B0000002000000030BCBDE8AE
:1089C000C08F2DE9F041044600251E461746880455
:1089D00004D405E039462020B0476D1C641EF9D54B
:1089E0002846BDE8F0812DE9F041044600251E46E9
:1089F0009046C80301D5302700E02027880404D51D
:108A000005E041463846B0476D1C641EF9D528463E
:108A1000BDE8F0810A68531C0B60107070470000BD
:108A200080F0010201210148FAF7C3BB00040048AD
:108A300082B0CDE9000121F0004001909DED000BD6
:108A400002B051EC100B704713B54FF0FF33012209
:108A500069460248FCF73CFA00981CBD406B0020B8
:108A600010B5002821D0114B0022001F196803E027
:108A7000814203D80A4649680029F9D152B11368E6
:108A8000841A9C4204D1006818441060104602E029
:108A9000506000E0186039B102680B1A934203D1AC
:108AA0000B681A4402604968416010BD1001002043
:108AB000FAF71AFEFDF7FCFFFDF78AFBFDF720FB36
:108AC000FDF746FCFDF7D4FBFDF7F6FAFDF7FCFBDE
:108AD00000F091F8014617A0FEF788FB1AA0FEF7F8
:108AE00085FB00F017FE002201211C48FAF761FB0C
:108AF000F8F732F81A48F9F735FF02211848F9F764
:108B000022FB3220FAF7D2F804213320FDF7BCFA19
:108B100014493320FCF753FF134C144920601148CB
:108B2000FCF754FF206000F06DF8FDF71FFB00F02C
:108B30007BF8FEE773746172745F7469636B202560
:108B40006C750D0A000000004D4C58393036343039
:108B50002032355F345F32340D0A000000040048D3
:108B6000106A0020262500200C000020A82B0020E1
:108B7000F0B50B30154D20F007010024144A0FE02A
:108B800003688B420BD38B4205D95E1A43184768A2
:108B9000C3E9006700E04368136002C004E0021DFF
:108BA00010680028ECD12046002802D1286808B1BE
:108BB0000020F0BD064A07481060074A121A22F04A
:108BC0000702C0E9002401202860D7E71401002033
:108BD000100100207C990020789B002010B5EFF355
:108BE000058111B16FF0050403E0002408B100F025
:108BF00007FF204610BDEFF3058008B101F000BC6F
:108C000001F0F8BBEFF3058010B16FF0050070477D
:108C10000448016811B14FF0FF3070470121016035
:108C200000207047DC00002010B5EFF3058010B184
:108C30006FF0050010BD08480168012902D04FF00F
:108C4000FF3010BD054A002182F8141D0221016089
:108C500000F084FF002010BDDC0000200BE000E0ED
:108C600070B505464FF00004EFF3058050BB0DB121
:108C7000686800E00020C10701D0012600E000265E
:108C800000071FD46DB1D5E9021021B1502819D3C6
:108C90001EB1042002E020B114E0012001F0B4F87C
:108CA00005E00EB1042000E0012001F0A2F804006C
:108CB00008D00DB1296800E0002100F03FFE0EB1A0
:108CC00044F00104204670BDF8B5144603460E4634
:108CD0004FF00005EFF3058098BB93B39E423DD85B
:108CE0004CB1A0680028E06803D0502836D301209A
:108CF00002E008B132E00020012B05D010B3184685
:108D0000A26801F056F820E040B103200090002254
:108D100011460120A36801F0A5F804E00322002118
:108D2000012001F07EF8050018D086B100231A4614
:108D3000194601F00FF9012809D0284600F012FE6B
:108D400000250BE0184601F017F8050006D00CB11D
:108D5000216800E00021284600F0F0FD2846F8BD1B
:108D60002DE9FF410B464FF00005EFF30581039518
:108D700049BB40B38027182100244AB3166806B1C6
:108D8000344696691EB13146761E382E02D21679C7
:108D9000F60703D0002004B0BDE8F081566906B1A3
:108DA000B708D2F808C0BCF1000F0DD0D5685C2D13
:108DB00018D312693AB136B18DE806103A46214609
:108DC00001F0DEFA03900DE0D6685EB912694AB987
:108DD00003AACDE90012BAB2214601F0A1FA012896
:108DE00000D003950398D6E72DE9F041134C0F46C8
:108DF0000546E6682068001D00F0A2FC681C07D14B
:108E000037B12168BDE8F0410D48091D00F0E8BC0C
:108E100020683544B5424560216805D2A06BBDE8A5
:108E2000F041091D00F0C4BC606B091D00F0C0FCDE
:108E3000A06A854200D2A562BDE8F0818C000020C6
:108E4000907100202DE9F041054600F0D5FC2D4C35
:108E5000A068401CA06020682B4F10B1606930B33F
:108E60002BE02560A068012827D1002606EB8600AC
:108E700007EB800000F08EFC761C382EF6D32348DA
:108E800000F088FC2148143000F084FC1F48283092
:108E900000F080FC1D483C3000F07CFC1B4850304A
:108EA00000F078FC194860631430A06305E0206886
:108EB000E96AC06A884200D82560606A401C606226
:108EC0006864E86A2169884200D9206100EB80006B
:108ED00007EB8000291D00F083FC00F0ADFC606909
:108EE00000280CD02068E96AC06A884207D2084985
:108EF0004FF080500860BFF34F8FBFF36F8FBDE816
:108F0000F08100008C000020E06C00204071002007
:108F100004ED00E038B500F06FFC104C2068C8B9D3
:108F20000F4800F037FC0E48143000F033FC0C48BA
:108F3000E060143020610A4B0020F03B009003F108
:108F4000500210210A2000F08DFF206010B105A111
:108F500000F0F4FCBDE8384000F06EBCC800002012
:108F600094720020546D72510000000030B4026C05
:108F70000B46002A0BD0C1681144C1608468A1422D
:108F800001D30168C16030BC1846F7F7BFB930BCE7
:108F900070472DE9F041856B174604460026026CA8
:108FA00082B1C7B1E068F7F7B1F9E168206C091A3E
:108FB000E1602268914202D2A168081AE060022FA3
:108FC00016D017E02068A8B9A06801F085FA064617
:108FD0000020A0600EE06068F7F798F9216C6068E7
:108FE00008446060A168884204D32068606001E0A2
:108FF00005B16D1E6D1CA5633046BDE8F08110B54E
:10900000044690F8590058B101280CD002280FD01E
:10901000502080F31188BFF34F8FBFF36F8FFEE7AF
:10902000206B00F01DFC2046BDE8104000F018BC8D
:1090300010BD000010484FF40051420706D0C01D7B
:109040000D4920F00700411AC1F500510B4A0023D9
:109050000144C2E900030839183A21F00701116000
:109060004B600B600B1AC0E9001393604FF0004097
:10907000536050617047000074790020F8000020B0
:10908000144E154CA6F29C474FF08058DFF84C90D8
:1090900012E000BF00F0B0FBF068C568281D00F0CA
:1090A0004FFBA068401EA0606068401E606000F03A
:1090B000C3FB2846FFF7A3FF60680028EAD13868A1
:1090C0000128F9D9C9F80080BFF34F8FBFF36F8F24
:1090D000F2E700007C7100208C00002004ED00E02D
:1090E000002807D00021816001600B460A46C1605C
:1090F00000F030BF7047000070B51D46049C51B1B0
:10910000C4F80020C4E90F010121204600F0DEFE72
:1091100084F84C5070BD2460F4E700002DE9F05F46
:109120008846DDE90B941546834691009A460A9ECF
:10913000A522206BF7F7FCF86FF00301206B01EB21
:109140008501084420F00707780707D0502080F3F6
:109150001188BFF34F8FBFF36F8FFEE70025B8F183
:10916000000F0FD05FF00000221818F8001082F8EE
:10917000341018F8001011B1401C1028F4D384F8F2
:10918000435001E084F83450382E00D33726E6628D
:10919000C4E91365201D00F008FB04F1180000F07D
:1091A00004FB2461C6F138006462A061656584F83F
:1091B000585052465946384600F05EFA2060B9F1E0
:1091C000000F01D0C9F8004000F000B830BCBDE885
:1091D000C09F000030B5114900E011460A68824284
:1091E000FBD34B685C18844203D140681844486044
:1091F000084643681C18944209D1084C183C24685E
:10920000A24209D052681A4442600A681268026099
:10921000814200D0086030BD0460F9E7F80000200A
:1092200070B5002441600B4D0061914206D8D11AFF
:109230008269914206D2011D286907E09A4203D251
:10924000994201D3012403E0011DE86800F0B0FA5F
:10925000204670BDC800002010B5044600F0CCFACE
:10926000A06B28B15FF0000400F0E6FA204610BDC4
:109270000124F9E730B589B03C4D6EE00498002830
:1092800006DADDE90601059A90470498002864DBB8
:10929000069C606910B1201D00F052FA03A800F08E
:1092A000D7F8024604980A2857D2DFE800F00505EF
:1092B000052D334A05052D3394F8280040F00100B0
:1092C00084F828000599A069059B01442046FFF712
:1092D000A7FF68B3216A2046884794F82800400712
:1092E0003BD5002000900598A1690023421819463B
:1092F000204601F0FBF9D8B9502080F31188BFF364
:109300004F8FBFF36F8FFEE714F8280F20F0010096
:10931000207022E094F8280040F0010084F8280032
:109320000598A06128B1811813462046FFF778FF01
:1093300013E0502080F31188BFF34F8FBFF36F8F7E
:10934000FEE794F82800810703D4204600F088FA4D
:1093500003E020F0010084F82800002204A9286816
:1093600000F008FF002889D109B030BDC8000020F6
:109370002DE9FC410F46054600F034FC01A800F041
:1093800067F80446019818B101F01EF9BDE8FC81A8
:10939000254EAFB130690068D0B30027291B3A468B
:1093A000306800F00BFB01F00FF90028EED11F49E7
:1093B0004FF080500860BFF34F8FBFF36F8FE5E72A
:1093C000A542EBD801F000F9F0682746C068C468F0
:1093D000201D00F0B5F994F82800410719D5A069BF
:1093E0002B4641193A462046FFF71AFFA8B1002044
:1093F0000346014600902A46204601F077F960B9FD
:10940000502080F31188BFF34F8FBFF36F8FFEE7BB
:1094100007E020F0010084F82800216A20468847F0
:10942000B4E70127BAE70000C800002004ED00E01F
:109430000648416B096829B1416BC968C968496828
:10944000816270474FF0FF31FAE700008C00002086
:1094500070B5054600F0CEFF064E0446B068844263
:1094600003D200F009F8012000E000202860204627
:10947000B46070BDC8000020F8B5194D20E0C06888
:10948000C4680668201D00F05BF9216A2046884701
:1094900094F82800400713D5A0693044B04206D99B
:1094A00024616060211DE86800F082F908E0002076
:1094B0000346014600903246204601F017F938B1C4
:1094C000E86801680029DAD12969C5E90310F8BD07
:1094D000502080F31188BFF34F8FBFF36F8FFEE7EB
:1094E000C800002008484068401C4FF0500080F33E
:1094F000118804D0BFF34F8FBFF36F8FFEE7BFF328
:109500004F8FBFF36F8FFEE700010020074CE0682C
:10951000016841B1C0680021D0F80000FFF728FFC2
:10952000FFF7A8FEF3E701210020F7E7C8000020BD
:109530002DE9F041044600F05FF994F9455004F13B
:10954000240609E0606A48B1304601F005F808B128
:1095500000F0CAFA6D1E6DB2002DF3DC4FF0FF363D
:1095600084F8456000F068F900F046F994F9445039
:1095700004F1100709E0206948B1384600F0ECFF1B
:1095800008B100F0B1FA6D1E6DB2002DF3DC84F865
:109590004460BDE8F04100F04FB900002DE9F04112
:1095A0000546002700F01EFB324E306808B9FFF771
:1095B00041FD706905424ED1C5B3083568070ED02C
:1095C00005F00700C0F108000544680707D05020E7
:1095D00080F31188BFF34F8FBFF36F8FFEE72DB37A
:1095E0007068854237D82348183001460C6801E07E
:1095F00020460C466168A94202D221680029F7D1B1
:1096000031688C4227D0076821680160606808379C
:10961000411B10290FD96019420708D0502080F350
:109620001188BFF34F8FBFF36F8FFEE713E04160E8
:109630006560FFF7CFFD61687068401A7060B268BE
:10964000904200D2B060706901430020C4E900017B
:10965000F068401CF06000F0B7FF780707D050209A
:1096600080F31188BFF34F8FBFF36F8FFEE738464B
:10967000BDE8F081E000002010B5031F4FF08074BA
:109680001C601B1F21F001011960191F044B0B60A6
:1096900014390A60091F6FF0020244380A6010BDD5
:1096A000E594000800B52DED048B83B041EC190B57
:1096B000F7F729F941EC180B18EE100A18EE901A7A
:1096C0008DED008B002818BF0120084320F00040DA
:1096D000C0F17F6000F1E040C00F14D019EE101A05
:1096E00019EE900A8DED009B002918BF0121084357
:1096F00020F00040C0F17F6000F1E040C00F04BFE7
:109700000120FEF731FD51EC180B03B0BDEC048BCA
:1097100000BD000010B509210748F6F710FE074804
:109720000068016841F010010160BDE810400922A5
:1097300001490248FBF7A0BB1C250020406B00201C
:10974000D0E9013201699A60D0E901235A604A6880
:10975000824201D182684A60002202610868401E8C
:109760000860086870470000034B036003F15C0069
:109770000860802010607047BC720020044B0360BA
:1097800003F15C0008604FF48070106070470000C7
:109790001875002000F108014FF0FF32C0E90112F6
:1097A000C1600161002101607047002101617047C3
:1097B00030B50B685A1C02D000F1080202E00269C1
:1097C00004E02246546825689D42FAD953684B60EC
:1097D00099608A60516008610168491C016030BD70
:1097E00042684A6093688B60936859609160086131
:1097F0000168491C01607047502080F31188BFF355
:109800004F8FBFF36F8F0A494868401C486001289A
:109810000CD10848006810F0FF0F07D0502080F3EB
:109820001188BFF34F8FBFF36F8FFEE770470000C3
:109830000001002004ED00E00849486828B1401EFE
:10984000486001D180F311887047502080F311885F
:10985000BFF34F8FBFF36F8FFEE7000000010020C2
:1098600070B500282AD0164DA0F108046068696917
:10987000084207D1502080F31188BFF34F8FBFF308
:109880006F8FFEE722683AB1502080F31188BFF352
:109890004F8FBFF36F8FFEE78843606000F0A2F93F
:1098A00060686968084468602046FFF793FC28698F
:1098B000401C2861BDE8704000F086BE70BD00000D
:1098C000E00000204FF0E0200021016181610549A6
:1098D0004FF47A720968B1FBF2F1491E4161072128
:1098E000016170478800002010B5F6F7B5FC1149FA
:1098F00010280ED300F1E02090F8F0030A7890428F
:1099000007D2502080F31188BFF34F8FBFF36F8FC2
:10991000FEE709480068896800F4E060884207D9DA
:10992000502080F31188BFF34F8FBFF36F8FFEE796
:1099300010BD0000000100200CED00E010B5084B48
:10994000002200BF53F832401CB1521C082AF9D340
:1099500010BD43F8321003EBC201486010BD000097
:10996000A06C002010B504000AD000F013F894F8A1
:10997000460000280CD12046BDE81040FFF770BF1C
:10998000502080F31188BFF34F8FBFF36F8FFEE736
:1099900010BD0000084A002102EBC1035B6883424E
:1099A00006D1002042F8310002EBC1014860704747
:1099B000491C0829F0D37047A06C002070B51546EB
:1099C0000E460446FFF718FF94F944100020491C86
:1099D00001D184F8440094F94510491C01D184F860
:1099E0004500FFF729FFA06B28B92A46314604F14C
:1099F000240000F097F82046BDE87040FFF798BDBE
:109A000010B5020014D00F48006B38B1502080F31D
:109A10001188BFF34F8FBFF36F8FFEE700F0E2F8BE
:109A200000211046FFF7E0F900F0CEFD002807D135
:109A300005494FF080500860BFF34F8FBFF36F8F21
:109A400010BD00008C00002004ED00E070B50D4654
:109A500004000BD095B11E4A106BB8B1502080F3B2
:109A60001188BFF34F8FBFF36F8FFEE7502080F355
:109A70001188BFF34F8FBFF36F8FFEE7502080F345
:109A80001188BFF34F8FBFF36F8FFEE700F0AAF886
:109A9000D26823685919934204D98B420AD991425A
:109AA00002D807E08B42FAD9881A21600021FFF71B
:109AB0009BF900E0216000F087FD002807D10549EF
:109AC0004FF080500860BFF34F8FBFF36F8F70BDB2
:109AD0008C00002004ED00E002490A6A0260C968B7
:109AE000416070478C00002001490120C861704727
:109AF0008C00002010B50C4650B109490968183196
:109B0000FFF756FE2046BDE810400121FFF76CB973
:109B1000502080F31188BFF34F8FBFF36F8FFEE7A4
:109B20008C00002070B514460D4668B10A490968DA
:109B30001831FFF755FE0CB14FF0FF35214628468E
:109B4000BDE87040FFF750B9502080F31188BFF393
:109B50004F8FBFF36F8FFEE78C00002030B587B0CA
:109B60000024039405AA04A903A80494FFF7FCFDAC
:109B7000DDE903010094CDE90110002315A1174888
:109B8000059A00F0FDFB164D0028E8621FD000F09A
:109B90007DFD012809D0401C19D1502080F3118887
:109BA000BFF34F8FBFF36F8FFEE7502080F3118814
:109BB000BFF34F8FBFF36F8F4FF0FF30A8620120CC
:109BC0006861EC6007B0BDE8304000F045B807B010
:109BD00030BD000049444C45000000008190000861
:109BE0008C0000200248016B491C01637047000093
:109BF0008C000020164810B5016B11B10121C16124
:109C000010BD0021C1610169124A01E0B9B1491ECC
:109C100001EB810352F82330002BF7D001EB8103D5
:109C200002EB830202F1080453685B685360A342AD
:109C300001D15B685360DA680260016110BD502099
:109C400080F31188BFF34F8FBFF36F8FFEE70000E3
:109C50008C000020E06C00201CB537480168374AB2
:109C6000914207D1502080F31188BFF34F8FBFF38B
:109C70006F8FFEE700683149491E884207D15020A6
:109C800080F31188BFF34F8FBFF36F8FFEE72C492E
:109C900008780190FF20087008788DF800009DF882
:109CA00000009DF8002000F0F000904207D0502006
:109CB00080F31188BFF34F8FBFF36F8FFEE79DF8DE
:109CC0000000204C00F0500020700720A06005E04C
:109CD0009DF8002052008DF80020401E9DF80020C5
:109CE0001206F5D4A060032807D0502080F3118815
:109CF000BFF34F8FBFF36F8FFEE74FF44070A0604C
:109D0000019808700C482030016841F4700101602E
:109D1000016841F070410160FFF7D4FD00206060F0
:109D2000F6F762FA0848016841F040410160F6F731
:109D300047FA00201CBD000000ED00E071C20F4199
:109D400000E400E00001002034EF00E010B55020F6
:109D500080F31188BFF34F8FBFF36F8F00F058FB74
:109D600018B104494FF080500860002080F311883A
:109D700010BD000004ED00E010B50C4648B184426F
:109D80000FD9502080F31188BFF34F8FBFF36F8F2F
:109D9000FEE7502080F31188BFF34F8FBFF36F8F22
:109DA000FEE70222002100F03CF8002800D0846386
:109DB00010BD38B50C4648B184420FD9502080F30D
:109DC0001188BFF34F8FBFF36F8FFEE7502080F3F2
:109DD0001188BFF34F8FBFF36F8FFEE70221134649
:109DE00000220091114600F03DF8002800D0846365
:109DF00038BD10B502460021012000F012F80446DB
:109E0000FFF76EF9204610BD38B50B4600220090D2
:109E10001146012000F026F80446FFF761F92046BC
:109E200038BDF8B517460E46050013D005FB06F001
:109E30005030FFF7B3FB04000AD0002084F846003E
:109E400004F150023B46314628460094FFF754F98E
:109E50002046F8BD502080F31188BFF34F8FBFF329
:109E60006F8FFEE738B5049D18B153B1CAB181B107
:109E700020E0502080F31188BFF34F8FBFF36F8F26
:109E8000FEE7502080F31188BFF34F8FBFF36F8F31
:109E9000FEE7502080F31188BFF34F8FBFF36F8F21
:109EA000FEE739B1502080F31188BFF34F8FBFF325
:109EB0006F8FFEE750241C46012384F846302B4662
:109EC0000094FFF719F9204638BD000070B50D4623
:109ED000040025D0FFF790FCD4E90F20216802FB95
:109EE0000011A1600021A163216861600A46D4E9E4
:109EF0000F01401E00FB0121E16021464FF0FF30C1
:109F000001F8440F487004F110008DB1FFF742FCD6
:109F100004F12400FFF73EFCFFF78EFC012070BD2A
:109F2000502080F31188BFF34F8FBFF36F8FFEE790
:109F300021690029F0D000F00FFB0028ECD0044983
:109F40004FF080500860BFF34F8FBFF36F8FE3E790
:109F500004ED00E02DE9FF4782B01D468A464FF030
:109F60000008040003D0BAF1000F08D011E050201F
:109F700080F31188BFF34F8FBFF36F8FFEE7206C24
:109F800038B1502080F31188BFF34F8FBFF36F8F2C
:109F9000FEE7022D0AD1E06B012807D0502080F3A4
:109FA0001188BFF34F8FBFF36F8FFEE700F014FAF5
:109FB0003F4F4FF000094FF0805648B9049838B130
:109FC000502080F31188BFF34F8FBFF36F8FFEE7F0
:109FD000FFF712FCA06BE16B884207D3022D05D07E
:109FE0000498D0B1B8F1000F1AD01EE02A465146AD
:109FF0002046FEF7CEFF616A19B104F1240000F09B
:10A00000ABFA20B13E60BFF34F8FBFF36F8FFFF706
:10A0100013FC012006B0BDE8F087FFF70DFC22E03D
:10A020006846FFF759FD4FF00108FFF705FCFFF701
:10A03000D9FDFFF7E1FB94F94400401C01D184F8FD
:10A04000449094F94500401C01D184F84590FFF7F5
:10A05000F3FB04A9684600F029F930B12046FFF768
:10A0600067FA00F0B1FA0020D4E7FFF7C5FBA06B58
:10A07000E16B884213D1FFF7DFFB04F11000049974
:10A08000FFF738FD2046FFF753FA00F09DFA00284D
:10A090009ED13E60BFF34F8FBFF36F8F98E7FFF7FE
:10A0A000CBFB2046FFF744FA00F08EFA90E7000061
:10A0B00004ED00E02DE9F0471F4690468946040074
:10A0C00003D0B9F1000F08D011E0502080F31188BF
:10A0D000BFF34F8FBFF36F8FFEE7206C38B1502076
:10A0E00080F31188BFF34F8FBFF36F8FFEE7022F0E
:10A0F0000AD1E06B012807D0502080F31188BFF30C
:10A100004F8FBFF36F8FFEE7FFF7EEFB5020EFF3AB
:10A11000118680F31188BFF34F8FBFF36F8FA06B51
:10A12000E16B884206D3022F04D0002086F3118809
:10A13000BDE8F08794F94550A06B3A464946204661
:10A14000FEF727FF681C04D06D1C84F845500120E1
:10A15000ECE7606A0028FAD004F1240000F0FCF972
:10A160000028F4D0B8F1000FF1D00121C8F8001098
:10A17000EDE700002DE9F747002683B08A4604008A
:10A1800003D0BAF1000F08D011E0502080F31188FD
:10A19000BFF34F8FBFF36F8FFEE7206C38B15020B5
:10A1A00080F31188BFF34F8FBFF36F8FFEE700F08E
:10A1B00013F9DFF8F4804FF000094FF0805748B9E9
:10A1C000059838B1502080F31188BFF34F8FBFF34B
:10A1D0006F8FFEE7FFF710FBA56BC5B15146204618
:10A1E000FEF7C4FE6D1EA563206950B104F1100096
:10A1F00000F0B2F928B1C8F80070BFF34F8FBFF379
:10A200006F8FFFF719FB012006B0BDE8F0870598B6
:10A2100008B11EB106E0FFF70FFB27E06846FFF725
:10A220005BFC0126FFF708FBFFF7DCFCFFF7E4FA15
:10A2300094F94400401C01D184F8449094F94500FD
:10A24000401C01D184F84590FFF7F6FA05A968464D
:10A2500000F02CF8002820460AD0FFF769F900F03A
:10A26000B3F92046FEF7F8FF0028B3D00020CBE773
:10A27000FEF7F2FF90B104F124000599FFF73AFCD4
:10A280002046FFF755F900F09FF90028A2D1C8F841
:10A290000070BFF34F8FBFF36F8F9BE72046FFF730
:10A2A00047F900F091F995E704ED00E02DE9F04160
:10A2B0000C46050011D0C4B1FFF79EFA174BDA68BF
:10A2C0006E682068911B471C17D02F681B6A9F423D
:10A2D00019D0964217D8012410E0502080F311883D
:10A2E000BFF34F8FBFF36F8FFEE7502080F31188CD
:10A2F000BFF34F8FBFF36F8FFEE70024FFF79CFA89
:10A300002046BDE8F081884205D9401A20602846E1
:10A31000FFF7E2FBF1E700202060DCE78C00002083
:10A320002DE9FF5F8346DDE90E87994616468A468A
:10A330009000FFF733F905001CD05C20FFF72EF9E1
:10A34000040014D00020256384F85900CDE90240B0
:10A35000CDE900874B46324651465846FEF7DEFEB1
:10A360002046FEF76FFD012004B000F006B8284635
:10A37000FFF776FA4FF0FF30F6E730BCBDE8C09F3C
:10A38000F0B585B0DDE90B640A9DA6B1DCB15C27B0
:10A3900000972663022684F85960002604AFCDE9B1
:10A3A0000246CDE90057FEF7B9FE2046FEF74AFD0A
:10A3B000049805B0F0BD502080F31188BFF34F8F93
:10A3C000BFF36F8FFEE7502080F31188BFF34F8FEC
:10A3D000BFF36F8FFEE700000548416919B1006BBC
:10A3E00018B100207047012070470220704700001C
:10A3F0008C0000200148C068704700008C000020DD
:10A4000010B5FFF771FA0148C06810BD8C0000203C
:10A410002DE9F0412E4C0027206B28B1A069401C8B
:10A42000A0613846BDE8F081E668761CE66013D18D
:10A43000606B006838B1502080F31188BFF34F8FF4
:10A44000BFF36F8FFEE7606BA16B6163A063206A4F
:10A45000401C2062FEF7ECFFA06ADFF8788086429D
:10A4600009D3606B0068A0B1606BC068C56868689C
:10A47000864211D2A0622068C06A00EB800158F8C1
:10A480002100012800D90127E0690028C9D001274F
:10A49000C7E74FF0FF30EDE7281DFFF751F9A86A35
:10A4A00018B105F11800FFF74BF9E86A21698842F5
:10A4B00000D9206100EB800108EB8100291DFFF726
:10A4C0008FF9E86A2168C96A8842CAD30127C8E7B8
:10A4D0008C000020E06C002070B504004FF00001FB
:10A4E00033D01B4D2868844207D0502080F3118858
:10A4F000BFF34F8FBFF36F8FFEE7206D38B1401E63
:10A500002065E36CE26A9A421FD040B11DE0502002
:10A5100080F31188BFF34F8FBFF36F8FFEE7201DCD
:10A52000FFF70EF9E06CE062C0F13800A061E06A6C
:10A530002969884200D92861064900EB800001EBB7
:10A540008000211DFFF74CF90121084670BD000075
:10A550008C000020E06C002070B5C068C46854B165
:10A5600004F118000646FFF7EBF8144D286B50B1C4
:10A570003146134815E0502080F31188BFF34F8F08
:10A58000BFF36F8FFEE7201DFFF7DAF8E06A296955
:10A59000884200D928610B4900EB800001EB800064
:10A5A000211DFFF71DF9E06A2968C96A884202D9AE
:10A5B0000120E86170BD002070BD00008C0000200B
:10A5C00068710020E06C00202DE9F0472C4D00243C
:10A5D0002746286B38B1FFF70FF9286B401E286318
:10A5E000286B40B146E0502080F31188BFF34F8FB5
:10A5F000BFF36F8FFEE7A968224E0120D1B3A6F505
:10A60000916980463068E0B1F068C46804F11800D0
:10A61000FFF796F8201DFFF793F8E06A2969884252
:10A6200000D9286100EB800109EB8100211DFFF7B3
:10A63000D7F8E06A2968C96A8842E3D3C5F81C8064
:10A64000E0E70CB1FEF7F4FEAC694CB14FEA080646
:10A65000FFF7DEFE00B1EE61641EF9D10020A861B3
:10A66000E86938B10849012738070860BFF34F8F00
:10A67000BFF36F8FFFF7E0F83846BDE8F0870000C2
:10A680008C0000206871002004ED00E010B586B059
:10A69000FEF740FC114C2068B8B1002003900490F4
:10A6A00005AA04A903A8FFF769F8DDE90321022040
:10A6B0008DE8070000230AA10B48059AFFF760FE0A
:10A6C000606010B106B0012010BD502080F31188E9
:10A6D000BFF34F8FBFF36F8FFEE70000C80000206D
:10A6E000546D7220537663000D9500082DE9FF41EB
:10A6F0001E46134602000A9D4FF0000016D0144C6F
:10A700002768002F0FD0CDE900130292062917DA2F
:10A71000FFF762FE02284FF000030FD000226946C7
:10A720002068FFF717FC04B0BDE8F081502080F3EB
:10A730001188BFF34F8FBFF36F8FFEE72A46EEE716
:10A740000023324669463846FFF7B4FCEBE70000C9
:10A75000C800002018A90008000000000000000048
:10A7600000000000000000000004000018000000CD
:10A77000000000000000000028A900080000000000
:10A7800000000000000000000000000000040000C5
:10A7900028000000000000000000000048A9000898
:10A7A00000000000000000000000000000000000A9
:10A7B0000002000030000000000000000000000067
:10A7C00050A9000800000000000000000000000088
:10A7D00038A9000800000000000000000000000090
:10A7E0000000000000000000010203040607080941
:10A7F000A0860100400D0300801A060000350C0001
:10A8000040420F0080841E0000093D0000127A00C3
:10A810000024F40000366E010048E801006CDC0200
:10A820000000000001020304000000000000F03FEF
:10A83000000000000000F83F0000000000000000E1
:10A840000000004003B8E23F0000000000000000EC
:10A8500006D0CF43EBFD4C3E033333333333E33F7A
:10A86000FFAB6FDBB66DDB3F4D268F515555D53FA6
:10A8700001411DA96074D13F65DBC9934A86CD3F74
:10A88000EF4E454A287ECA3F3E5555555555C53F62
:10A8900093BDBE166CC166BF2CDE25AF6A56113F54
:10A8A000F16BD2C541BDBBBED0A4BE726937663E56
:10A8B00000000000000000004C6F616465642064CB
:10A8C0006174613A2066697273745F74687265734B
:10A8D000686F6C643D25752C207365636F6E645FD3
:10A8E0007468726573686F6C643D2575202C2064F4
:10A8F000656C61795F726563656976656456616CE4
:10A9000075653D2575202C456D697373697669748D
:10A91000793D25750A0000007265616454656D70AB
:10A920005461736B0000000073656E6454656D7054
:10A930005461736B0000000064617461526561646E
:10A940007953656D00000000436F6D6D6F6E000000
:10A95000646174614D757465780000007CA900081D
:10A96000000000201C0100004881000898AA00088F
:10A970001C0100205C9E00005881000800000000BF
:10A9800000000000000000000000000000000000C7
:10A9900000003C64015F00000000000000000000B7
:10A9A00000000000000000000000000000000000A7
:10A9B0000000000000000000000000000000000097
:10A9C0000000000000000000000000000000000087
:10A9D0000000000000000000010000001000000066
:10A9E0000000000000000000000000000000000067
:10A9F0000000000001000000000000000000000056
:10AA00000000000000093D00000000000000000000
:10AA10000000000000000000000000000000000036
:10AA20000000000000000000000000000000000026
:10AA30000000000000000000000000000000000016
:10AA40000000000000000000000000000000000006
:10AA500000000000000000000000000000000000F6
:10AA600000000000000000000000000000000000E6
:10AA700000000000000000000000000000000000D6
:10AA8000AAAAAAAA0000000000000000000000001E
:08AA90000000000000000000BE
:040000050800018D61
:00000001FF
